:1015790020002A2A2000202A2A002020416464729F
:101589006573733A20202025303458002020526595
:10159900766973696F6E3A202025730025303342CE
:1015A9006430302530336430323D3F0025303342DA
:1015B900640D0025303342643130253033643036D0
:1015C9002530366C640025303342643130253033A0
:1015D9006430332530336C640050312A3A20253980
:1015E9002E3245206D6261720050313A202531302A
:1015F9002E3245206D6261720050322A3A20253917
:101609002E3245206D6261720050323A2025313008
:101619002E3245206D626172004552524F523A2076
:10162900747572626F20636F6D6D2E2020004552B4
:10163900524F523A20666F72652076616363757501
:101649006D20004552524F523A206D61696E2076E5
:1016590061636375756D2000544D50204552524F9A
:10166900523A2025732020202000544D503A20253D
:10167900346420487A2C2025342E326620410052C9
:101689006D7020646F776E20544D503A2534642074
:10169900487A0050756D702073746174696F6E209B
:1016A9006F666620202020005374617274696E672A
:1016B90020666F72652070756D7020200050756D01
:1016C90070696E67206275666665722074616E6BFB
:1016D900200050756D70696E672072656369706965
:1016E900656E742020200046503000465031005667
:1016F900563000565631004856300048563100429F
:10170900563000425631004F4646004F4E20005594
:101719004E4C4F434B00204C4F434B200050554DEE
:10172900502D53544154494F4E002449643A207373
:1017390063735F313030315F70756D702E632034A3
:1017490031383820323030382D30342D3234203190
:10175900323A30313A31325A2072697474405053F6
:10176900492E434820240001340000004572726F5D
:1017790072000000010C0E000000000000000000D3
:101789000000000000000001320000005374617481
:10179900696F6E00010C0F00000000003F8000001F
:1017A9003F80000000000001320000004C6F636BB5
:1017B90065640000010C1000000000003F8000007B
:1017C9003F800000000000013200000056616320E4
:1017D9004F4B0000010C1100000000003F80000089
:1017E9003F80000000000001320000004D616E4D95
:1017F9006F646500010C1200000000003F800000CA
:101809003F8000000000000132000000466F726551
:1018190070756D70010C1300000000003F8000001E
:101829003F8000000000000132000000466F726531
:10183900766C7600010C1400000000003F80000067
:101849003F80000000000001320000004D61696E18
:10185900766C7600010C1500000000003F80000046
:101869003F800000000000013200000042797076DC
:101879006C760000010C1600000000003F8000009B
:101889003F800000000000013200000054757262C0
:101899006F206F6E010C1700000000003F800000F0
:1018A9003F8000000000000214000000526F7453D2
:1018B90070640000010C1800000000000000000026
:1018C900000000000000000406000001544D5063B0
:1018D90075720000010C1A000000000000000000F1
:1018E9000000000000000001320000005650206F87
:1018F9006E000000010C1E00000000000000000046
:101909000000000000000001320000005656206F60
:1019190070656E00010C1F0000000000000000004F
:10192900000000000000000132000000565620634C
:101939006C6F7365010C20000000000000000000BE
:101949000000000000000001320000004856206F2E
:1019590070656E00010C210000000000000000000D
:10196900000000000000000132000000485620631A
:101979006C6F7365010C220000000000000000007C
:101989000000000000000001320000004256206FF4
:1019990070656E00010C23000000000000000000CB
:1019A90000000000000000013200000042562063E0
:1019B9006C6F7365010C240000000000000000003A
:1019C900000000000000000416FD00014856000058
:1019D90000000000010C25000000000000000000CC
:1019E900000000000000000416FD0001565600002A
:1019F90000000000010C29000000000000000000A8
:101A090000000000000000021400000846696E533F
:101A190070640000010C2D000000000000000000AF
:101A290000000000000000020400000854696D6510
:101A39006F757400010C2F00000000004396000030
:101A49004120000000000002030000084650206306
:101A590079636C65010C31004120000044160000D7
:101A6900412000000000000416FD00095656206DB3
:101A790061780000010C33013F8000004120000023
:101A89003F8000000000000416FD00095656206D35
:101A9900696E0000010C37013DCCCCCD3F800000C0
:101AA9003DCCCCCD0000000416FD00094856207439
:101AB90068727368010C3B033A83126F3F80000020
:101AC9003A83126F000000041800000941444330B2
:101AD90000000000010C3F000000000000000000B1
:101AE90000000000000000041800000941444331CF
:101AF90000000000010C430000000000000000008D
:101B090000000000000000041800000941444332AD
:101B190000000000010C4700000000000000000068
:101B2900000000000000000418000009414443338C
:101B390000000000010C4B00000000000000000044
:101B4900000000000000000418000009414443346B
:101B590000000000010C4F00000000000000000020
:101B6900000000000000000418000009414443354A
:101B790000000000010C53000000000000000000FC
:101B89000000000000000004180000094144433629
:101B990000000000010C57000000000000000000D8
:101BA9000000000000000004180000094144433708
:101BB90000000000010C5B000000000000000000B4
:101BC900000000000000000418000009414F4653BE
:101BD90030000000010C5F03BDCCCCCD3DCCCCCD99
:101BE9003A83126F0000000418000009414F465360
:101BF90031000000010C6303BDCCCCCD3DCCCCCD74
:101C09003A83126F0000000418000009414F46533F
:101C190032000000010C6703BDCCCCCD3DCCCCCD4E
:101C29003A83126F0000000418000009414F46531F
:101C390033000000010C6B03BDCCCCCD3DCCCCCD29
:101C49003A83126F0000000418000009414F4653FF
:101C590034000000010C6F03BDCCCCCD3DCCCCCD04
:101C69003A83126F0000000418000009414F4653DF
:101C790035000000010C7303BDCCCCCD3DCCCCCDDF
:101C89003A83126F0000000418000009414F4653BF
:101C990036000000010C7703BDCCCCCD3DCCCCCDBA
:101CA9003A83126F0000000418000009414F46539F
:101CB90037000000010C7B03BDCCCCCD3DCCCCCD95
:101CC9003A83126F000000045D0000094147414951
:101CD9004E300000010C7F033F6666663F8CCCCD19
:101CE9003A83126F000000045D0000094147414931
:101CF9004E310000010C83033F6666663F8CCCCDF4
:101D09003A83126F000000045D0000094147414910
:101D19004E320000010C87033F6666663F8CCCCDCE
:101D29003A83126F000000045D00000941474149F0
:101D39004E330000010C8B033F6666663F8CCCCDA9
:101D49003A83126F000000045D00000941474149D0
:101D59004E340000010C8F033F6666663F8CCCCD84
:101D69003A83126F000000045D00000941474149B0
:101D79004E350000010C93033F6666663F8CCCCD5F
:101D89003A83126F000000045D0000094147414990
:101D99004E360000010C97033F6666663F8CCCCD3A
:101DA9003A83126F000000045D0000094147414970
:101DB9004E370000010C9B033F6666663F8CCCCD15
:101DC9003A83126F000000000000000000000000CC
:101DD90000000000000000000000000000000000FA
:071DE90000000000000000F3
:105A4000016C010308FF1770410CA301C113C114BD
:105A5000C115C116C117C118410C0800410C09FF3E
:075A6000440C0A00000000E5
:10435C00E4F584F5BA75BCE075E880F5D1F58475A3
:10436C00D102F58475D48075840175D48075840F61
:10437C0075A4F575A5BF75A6FF75A7FFEF700302B1
:10438C004411E4900C0FF0A3F0A3F0A3F0F54174EA
:10439C00132541F582E4340CF583E4F00541E54145
:1043AC00B404ECE4F541E54125E025E0245FF58219
:1043BC00E4340CF583120A5600000000E54125E0B8
:1043CC0025E0247FF582E4340CF583120A563F80F5
:1043DC0000000541E541B408CD900C2FE4F0A37426
:1043EC003CF0A3E4F0A37414F0A3120A564080002E
:1043FC0000900C37120A563ECCCCCD900C3B120AD6
:10440C00563A83126FE4F541AF4112585A0541E513
:10441C0041C3941440F27D037F0112595075480733
:10442C007547B27546017545007D067F177E0012F3
:10443C004C127B017A0D792E7F3B7E011248D67B84
:10444C00017A0D792E124FE2900C2DEEF0A3EFF0C5
:10445C00E4FDFF125E64E4F5417B007A0079921270
:10446C005E4F7C007D0212080CC374079FFFE49E14
:10447C00FEC3E5419FEE6480F8748098500D7BFF7D
:10448C007A157979125D09054180CE7BFF7A157911
:10449C007B125D097B007A007992125D097BFF7AB1
:1044AC0015797F125D097D01E4FF125E647BFF7A52
:1044BC00157983788CE6F54C08E6F54D1234F87DC9
:1044CC0002E4FF125E64782E7C0D7D017BFF7A176F
:1044DC007948120BB97B017A0D792E7D20125E1D65
:1044EC00E41207C6754C01754D0D754E2E7BFF7A87
:0B44FC001579951234F8E4900C0EF0D6
:014507002291
:10585A00150EA80EEFF6A80EE624FC6018146020B8
:10586A0014602814603024047035900C11E024FF71
:10587A00B392B692B7900C13E024FFB392B0801F94
:10588A00900C14E024FFB392B18014900C15E0241C
:10589A00FFB392B28009900C16E024FFB392B305CD
:0258AA000E22CC
:050003008F377F002291
:105C5A008B378A388939120780AB3AAA3BA93C129A
:105C6A0007C6AB37AA38A939900001120799AB3A8F
:0D5C7A00AA3BA93C9000011207D87F02222E
:0A4508008E3D8F3E8B3F8A408941B3
:10451200E4F584E53E540FF5BB75BCE075480475BF
:104522004900E4F545F544F543F542F546F547C340
:10453200E5479549E5469548503AC2AFE4F584C24D
:10454200EDD2EC30EDFDD2AFAFBFEFFEADBEEDFF71
:10455200E4FCFDE5452FF545E5443EF544ED3543E4
:10456200F543EC3542F5421252690547E54770BF03
:10457200054680BBAF45AE44AD43AC427806120956
:104582003F8F458E448D438C42C3E53E9402E53D08
:10459200648094805024E41203B1E4FBFA798078B9
:1045A200471202A7E4FBFA79A0784112019EE4FBCC
:1045B200FA792078C11200AD8020AF45AE44AD43F8
:1045C200AC42E41203B1E4FBFA798078471202A705
:1045D200E4FBFA7920784112019E8F4D8E4C8D4B6F
:1045E2008C4AAF4DAE4CAD4BAC4AECC0E0EDC0E0F6
:1045F200EEC0E0EFC0E0E53EAE3D7802C333CE331D
:10460200CED8F9245FF582740C3EF583E0F8A3E07E
:10461200F9A3E0FAA3E0FBD0E0FFD0E0FED0E0FD9A
:10462200D0E0FC1200A98F4D8E4C8D4B8C4AECC011
:10463200E0EDC0E0EEC0E0EFC0E0E53EAE3D780266
:10464200C333CE33CED8F9247FF582740C3EF58382
:10465200E0F8A3E0F9A3E0FAA3E0FBD0E0FFD0E0AA
:10466200FED0E0FDD0E0FC12019E8F4D8E4C8D4BB2
:0F4672008C4AC2AFAB3FAA40A9411209A2D2AFF6
:014681002216
:104E6F00C297D296D2957F017E0012562CC295A280
:104E7F0096E433900C20F0D2977F017E0012562CCF
:104E8F00C2977F017E0012562CA296E433900C211C
:104E9F00F0D2977F017E0012562CC2977F017E00C1
:104EAF0012562CA296E433900C1EF0D2977F017EFF
:104EBF000012562CC2977F017E0012562CA296E448
:104ECF0033900C1FF0D2977F017E0012562CC297A1
:104EDF007F017E0012562CA296921CD2977F017EE4
:104EEF000012562CC2977F017E0012562CA296926A
:104EFF001BD2977F017E0012562CC2977F017E0036
:104F0F0012562CA296921AD2977F017E0012562C1F
:0E4F1F00C2977F017E0012562CA29692192294
:0848CE007B017A0D792E7E01B9
:0648D6008B428A43894475
:1048DC00754CFF754D15754EA5754F018E508F514A
:1048EC007B017A0D796E1234F2E4900D90F0900DFC
:1048FC008EF0900D8EE0FFC3940C501A746E2FF551
:10490C0082E4340DF583E0FF900D90E02FF0900DD4
:10491C008EE004F080DC754CFF754D15754EB5902E
:10492C000D90E0F54F7B017A0D797A1234F2E49018
:10493C000D8EF07B017A0D796E125E4F900D8EE02C
:10494C00FDC39FEE6480F87480985017746E2DF53B
:10495C0082E4340DF583E0FF125BAC900D8EE00425
:10496C00F080D0125DA37B017A0D796E754D147DAC
:10497C00201252F9900D8EEFF0D394024057900D07
:10498C0076E024D075F00AA4FFA3E024D02F900D7C
:10499C0091F0E4900D8FF0900D91E0FF900D8FE071
:1049AC00FEC39F502174782EF582E4340DF583E01C
:1049BC00AB42AA43A9448E827583001207D8900D8E
:1049CC008FE004F080D1AB42AA43A9448E82758358
:0749DC0000E40207D87F0090
:0149E30022B1
:074C0B00F5457D067F0CFE5C
:064C12008E428F438D4429
:104C1800E544B4060B754CFF754D15754EBC800EFA
:104C2800E544B40327754CFF754D15754ECF754F88
:104C380001854250854351854855854754854653DB
:104C48008545527B017A0D796E1234F2E4900D8F0E
:104C5800F0900D8EF0900D8EE0FFC39410501A74F2
:104C68006E2FF582E4340DF583E0FF900D8FE02F71
:104C7800F0900D8EE004F080DC754CFF754D1575D5
:104C88004EB5900D8FE0F54F7B017A0D797E123489
:104C9800F2E4900D8EF07B017A0D796E125E4F90E2
:104CA8000D8EE0FDC39FEE6480F8748098501774F1
:104CB8006E2DF582E4340DF583E0FF125BAC900DA8
:104CC8008EE004F080D0125DA37B017A0D796E75B9
:0C4CD8004D327D201252F9900D8EEFF04D
:014CE40022AD
:0B000E00900C0EF0E4FF125EF3E4FF24
:0A001900900C13EFF07F0402585A18
:0A5EF300900C14EFF07F0502585ADE
:0A5EFD00900C15EFF07F0602585AD2
:075E9E00E4FF125EFDE4FFCA
:0A5EA500900C16EFF07F0702585A28
:100CD100300803125ECFE4FDFF125E64900C13E056
:100CE100600CA3E060087BFF7A1579E280067BFF48
:100CF1007A1579F2900C29E0FCA3E0FDA3E0FEA3B4
:100D0100E0F54F8E4E8D4D8C4C1234F87D01E4FF91
:100D1100125E64900C17E06012900C15E07004A351
:100D2100E060087BFF7A16790280067BFF7A1679EC
:100D310012900C25E0FCA3E0FDA3E0FEA3E0F54F3B
:100D41008E4E8D4D8C4C1234F87D02E4FF125E64A0
:100D5100900C0EE030E0097BFF7A167922020E3CFE
:100D6100900C0EE030E1097BFF7A167937020E3CD8
:100D7100900C0EE030E2097BFF7A16794C020E3CB2
:100D8100900C0EE030E312754C01754D0C754EA4BC
:100D91007BFF7A167961020E3C900C12E060257B94
:100DA100FF7A167973900C18E0F54CA3E0F54DA38A
:100DB100E0FCA3E0FDA3E0FEA3E0F5518E508D4FD2
:100DC1008C4E8077900CA3E0B40122900C18E0FEC9
:100DD100A3E0FFD3940AEE94007BFF400A7A1679D0
:100DE100888E4C8F4D80547A16799C804E900CA33E
:100DF100E0B402087BFF7A1679B1803F900CA3E042
:100E0100B403087BFF7A1679C68030900CA3E07B8F
:100E1100FFB404067A1679DB80217A167973900C77
:100E210018E0F54CA3E0F54DA3E0FCA3E0FDA3E041
:100E3100FEA3E0F5518E508D4F8C4E1234F8900C7C
:100E410012E07003020F3D7D03E4FF125E64900C1B
:100E510013E07BFF60067A1679F080047A1679F444
:100E61001234F87D037F05125E64900C14E07BFF61
:100E710060067A1679F880047A1679FC1234F87DC6
:100E8100037F0B125E64900C15E07BFF60067A17FE
:100E9100790080047A1779041234F87D037F1012E7
:100EA1005E64900C16E07BFF60067A177908800477
:100EB1007A17790C1234F8301914201311900C138D
:100EC100E070047F0180027F00900C13EFF0301A74
:100ED10014201411900C14E070047F0180027F0033
:100EE100900C14EFF0301B14201511900C15E070CC
:100EF100047F0180027F00900C15EFF0301C14205C
:100F01001611900C16E070047F0180027F00900C96
:100F110016EFF07F0412585A0F12585A0F12585AEE
:100F21000F12585A201B03020FAF201C03020FAFF0
:100F3100124E6F201BFA201CF77F01227D03E4FF74
:100F4100125E64900C0FE07BFF60067A17791080C7
:100F5100047A1779141234F87D037F04125E6490C9
:100F61000C10E07BFF60067A17791880047A1779F4
:100F71001F1234F8301914201311900C0FE0700473
:100F81007F0180027F00900C0FEFF0301A142014C3
:100F910011900C10E070047F0180027F00900C1012
:100FA100EFF0200809201C063016037F0122A21948
:100FB1009213A21A9214A21B9215A21C9216900CC3
:100FC1000FE06024201721E4F548F547F546124C5F
:100FD1000B125E9E7F01120019900CA37402F01295
:100FE1005F07900C9F120A31900CA3E0B4024312E8
:100FF1005F07C8ECC8C9EDC9CAEECACBEFCB900CEC
:101001009FE0FCA3E0FDA3E0FEA3E024F4FFEE34A7
:1010110001FEE43DFDE43CFCD312092E40147F01A6
:10102100125EF3125F07900C9F120A31900CA374A9
:1010310003F0900CA3E0B4033A125F07C8ECC8C9EF
:10104100EDC9CAEECACBEFCB900C9FE0FCA3E0FD4B
:10105100A3E0FEA3E02490FFEE345FFEE43DFDE457
:101061003CFCD312092E400B900CA3740AF07402BD
:1010710012000E900CA3E064037076FFFE7D807C6D
:101081003F900C29E0F8A3E0F9A3E0FAA3E0FB12FA
:101091000344505DE4FFFE7D807C3F900C25E0F829
:1010A100A3E0F9A3E0FAA3E0FB120344500280326B
:1010B100900C10E0601B900C177401F0FF125EF3AE
:1010C100125F07900C9F120A31900CA37405F080F7
:1010D10020E4FF125EF37FD07E07125CDE7F0112F7
:1010E1005EA5125F07900C9F120A31900CA3740445
:1010F100F0900CA3E064047067D3900C30E094008E
:10110100900C2FE094004058125F07ECC0E0EDC056
:10111100E0EEC0E0EFC0E0900C2FE0FEA3E0FFE4C2
:10112100FCFD7B707A17F9F81208BB900C9FE0F870
:10113100A3E0F9A3E0FAA3E02FFBEA3EFAE93DF9C7
:10114100E83CF8D0E0FFD0E0FED0E0FDD0E0FCC309
:1011510012092E500B900CA3740AF0740412000EA5
:10116100900CA3E0B4041FE4FFFE7D807C3F900C53
:1011710025E0F8A3E0F9A3E0FAA3E0FB1203445051
:10118100057F01125EF3900CA3E0B40449E4FFFE75
:101191007D807C3F900C25E0F8A3E0F9A3E0FAA361
:1011A100E0FB120344502FE4FFFE7D807C3F900C56
:1011B10029E0F8A3E0F9A3E0FAA3E0FB120344500D
:1011C10015900C177401F0125F07900C9F120A31F1
:1011D100900CA37405F0900CA3E0FF64056014EF7C
:1011E1006406600FEF6407600AEF64086005EF644E
:1011F100097041E4FFFE7D807C40900C25E0F8A35E
:10120100E0F9A3E0FAA3E0FB120344602740259034
:101211000C10E0701FFF125EFDE4FF125EF3E4901C
:101221000C17F0900C0FE0600BC217900CA3740127
:10123100F07F0022900C10E060030212E4900CA3F6
:10124100E0640560030212E4900C2DE0FCA3E0FDD4
:10125100E41203B67BCD7ACC794C783F12019EEC37
:10126100C0E0EDC0E0EEC0E0EFC0E0900C18E0FCA3
:10127100A3E0FDE41203B6C8ECC8C9EDC9CAEECAC1
:10128100CBEFCBD0E0FFD0E0FED0E0FDD0E0FC1210
:101291000344604F404DE4FFFE7D807C3F900C2570
:1012A100E0F8A3E0F9A3E0FAA3E0FB120344503312
:1012B100E4FFFE7D807C3F900C29E0F8A3E0F9A3D8
:1012C100E0FAA3E0FB1203445019E4FF125EA57F8C
:1012D10001125EFD125F07900C9F120A31900CA360
:1012E1007406F0900C10E06401600302136E900C20
:1012F100A3E064057077900C2DE0FCA3E0FDE412FF
:1013010003B67BCD7ACC794C783F12019EECC0E0DC
:10131100EDC0E0EEC0E0EFC0E0900C18E0FCA3E00F
:10132100FDE41203B6C8ECC8C9EDC9CAEECACBEFD9
:10133100CBD0E0FFD0E0FED0E0FDD0E0FC120344D2
:10134100602B4029E4FFFE7D807C3F900C29E0F872
:10135100A3E0F9A3E0FAA3E0FB120344500F125FEC
:1013610007900C9F120A31900CA37406F0900CA305
:10137100E0640660030213F8125F07ECC0E0EDC001
:10138100E0EEC0E0EFC0E0900C31E0FEA3E0FF7CB6
:10139100007D641207FAE4FD900C9FE0F8A3E0F9E8
:1013A100A3E0FAA3E02FFBEA3EFAED39F9EC38F8B5
:1013B100D0E0FFD0E0FED0E0FDD0E0FCC312092E6A
:1013C1005035900C37E0FCA3E0FDA3E0FEA3E0FF65
:1013D100900C29E0F8A3E0F9A3E0FAA3E0FB1203E3
:1013E100445014E4FF125EF3900CA37409F0125FF1
:1013F10007900C9F120A31900CA3E0B4093A125FD6
:1014010007C8ECC8C9EDC9CAEECACBEFCB900C9F97
:10141100E0FCA3E0FDA3E0FEA3E0242CFFEE3401F9
:10142100FEE43DFDE43CFCD312092E400BE4FF1227
:101431000019900CA37407F0900CA3E0B407379047
:101441000C33E0FCA3E0FDA3E0FEA3E0FF900C2938
:10145100E0F8A3E0F9A3E0FAA3E0FB12034460166D
:1014610040147F01120019900CA37408F0125F0759
:10147100900C9F120A31900CA3E0B4083A125F0756
:10148100C8ECC8C9EDC9CAEECACBEFCB900C9FE03E
:10149100FCA3E0FDA3E0FEA3E024E8FFEE3403FE9D
:1014A100E43DFDE43CFCD312092E400B7F01125EAA
:1014B100F3900CA37406F0900C3BE0FCA3E0FDA3B9
:1014C100E0FEA3E0FF900C25E0F8A3E0F9A3E0FA29
:1014D100A3E0FB120344600250047F0180027F00FD
:1014E100900C11EFF07F0312585A900C0FE0703CF2
:1014F100301739FF125EF3125E9EE4FF120019E409
:10150100900C17F07548077547B2754601124C0BE0
:10151100E4F548F547F546F5457D037F1EFE124C7F
:1015210012900CA37401F0E4900C0EF0900C10E0FA
:101531006006201803125E9E900C10E0702930188E
:1015410026900C0FE06020125F07900C9F120A3169
:10155100900CA37403F07F011200197FE87E03123F
:101561005CDE7F01125EF3900C0FE024FF9217A363
:07157100E024FF92187F0047
:011578002250
:10412900900C08E075F004A4243FF9740C35F0FAFA
:104139007B01E0FF7E00124508900C08E0703D7F8E
:10414900427E607DD57C3F900C3FE0F8A3E0F9A367
:10415900E0FAA3E0FB12019E7BAE7A47793578C17C
:104169001200AD8F448E438D428C417F007E007DCD
:10417900207C411247B7900C25120A31900C08E0B7
:10418900B40131E4FFFE7DB07CC0900C43E0F8A39C
:10419900E0F9A3E0FAA3E0FB1200AD8F448E438D52
:1041A900428C417F007E007D207C411247B7900CF4
:1041B90029120A31900C08E0B40527E4FFFE7DA01E
:1041C9007C40900C53E0F8A3E0F9A3E0FAA3E0FBEC
:1041D900120344600640047F0180027F00900C2294
:1041E900EFF0900C08E0B40627E4FFFE7DA07C40C8
:1041F900900C57E0F8A3E0F9A3E0FAA3E0FB12035F
:1042090044600640047F0180027F00900C23EFF098
:10421900900C08E0B40727E4FFFE7DA07C40900CD9
:104229005BE0F8A3E0F9A3E0FAA3E0FB1203446022
:104239000640047F0180027F00900C24EFF0900C6F
:1042490008E0045407F0124E6F125F07C8ECC8C9A2
:10425900EDC9CAEECACBEFCB900C0AE0FCA3E0FD96
:10426900A3E0FEA3E02464FFE43EFEE43DFDE43C5C
:10427900FCD312092E5003024359900C09E0FF9018
:104289000C17E0FE6F602BEE600A7F077EB27D019E
:104299007C008005E4FFFEFDFC8F488E478D468C2F
:1042A900457D067F0A7E00124C12900C17E0900C97
:1042B90009F07F351248CEEF7003024349900C0E86
:1042C900E054FEF07B017A0D792E124FE2900C1822
:1042D900EEF0A3EFF07F361248CEEF60237B017A30
:1042E9000D792E124FE2CCEECCCDEFCDEC1203B608
:1042F900E4FBFA79C878421202A7900C1A120A3123
:104309007B017A0D792E7F2F7E011248D6EF603717
:104319007B017A0D792E124FE2EF4E900C0E60154B
:10432900E04408F078A47C0C7D017B017A0D792E9C
:10433900120BB98012E054F7F0E4900CA4F0800756
:10434900900C0EE04401F0125F07900C0A120A313A
:03435900022D979B
:105CB30020202020557067726164696E6700202080
:105CC30020204669726D776172652E2E2E00245254
:0B5CD30065763A20343136352024007D
:10390500E47880F6125E7875840F75E104E4F5E2DB
:1039150075E344F58475B7B075840F758A83F5979B
:10392500438901758D01758F01758E04F53FF5404D
:103935000540E5407002053F640F453F70F243893D
:1039450002E4F53FF540AE3FAF40E4FCFD7B507A25
:10395500C3F9F8D3120918400FE58920E40A054098
:10396500E54070E2053F80DE759702125DC2E4FF17
:10397500125DE1E4F53FF5407D01AF40125D330591
:1039850040E5407002053FC39403E53F940040E8DD
:10399500E4F520C228C226C22CC22BC22A7880F6A2
:1039A500C28508F67885F618F6788AF6F53FF5406B
:1039B50074AE2540F582E4340CF583E4F00540E56A
:1039C500407002053F6440453F70E5E4F53FF54032
:1039D50074EE2540F582E4340CF583E4F00540E50A
:1039E500407002053F6440453F70E5E4F584E5EF2E
:1039F50020E10CE5EF5408D394004003D38001C3C4
:103A050092037D08E4FF125950125527E47889F690
:103A15007882F6AB08AA09A90A7882E6FF75F02034
:103A2500A4F58285F083120799FE788926F6EE6063
:103A35000578820680DDEFD394004030AB08AA09F3
:103A4500A90A90000D120A97120780FF74551207F4
:103A5500C612078064556002D22A74AA1207C612DC
:103A6500078064AA6002D22AEF1207C6E4F584E54E
:103A7500EF5402D3940040047F018002E4FF124C0E
:103A8500E58F3EE53E20E036C22774FF788CF608C8
:103A9500F608F608F67E007F107D007B007A007937
:103AA50092120BD67546FF7547177548267549005E
:103AB500754A107B007A0079921258FE8002D2274F
:103AC500905CD8E493FF3395E0FEEF24D0FFEE340D
:103AD500FFFE7C007D641207FAAA06AB07905CD74F
:103AE500E493FF3395E0FEEF24D0FFEE34FFFE7C38
:103AF500037DE81207FAEF2BFBEE3AFA905CD9E466
:103B050093FF3395E0FEEF24D0FFEE34FFFE7C00FB
:103B15007D0A1207FAEF2BFFEE3AFEA3E493FD337D
:103B250095E0FCED24D0FDEC34FFCD2F7891F6ED3A
:103B35003E18F6E53E30E103023BE3E4F53FF54090
:103B4500E540AE3F7805C333CE33CED8F9FFAB0899
:103B5500AA09A90AF5828E831207996078E92FF9D7
:103B6500EA3EFA90000412079920E25EE4F53DE58D
:103B75003DC3786C965053E540AE3F7805C333CED0
:103B850033CED8F9AB08AA09A90AF5828E831207A4
:103B950099FF7E00C006C0077D00E540AE3F780571
:103BA500C333CE33CED8F929F9EA3EFA90000D1287
:103BB5000A977889E6853DF0A429F9EA35F0FAD027
:103BC50007D006120BD6053D80A50540E5407002DD
:103BD500053F023B457F0112435CC2298007E4FF94
:103BE50012435CD229E4F53FF5407A007B967D03CC
:103BF500AF401255A10540E5407002053FC394034F
:063C0500E53F940040E4DD
:013C0B002296
:055F1B00788AE6FF2278
:03002300024AF896
:104AF800C0E0C0F0C083C082C0D075D000C000C084
:104B080001C002C003C004C005C006C00730993EFA
:104B1800C2997885067985E77881667015F6788573
:014B2800F696
:0D4B290075260A75271300D527FCD526F642
:044B3600C285801C98
:0D4B3A0075261475271300D527FCD526F627
:104B47007885E624EEF582E4340CF583E0F59920C8
:104B57009803024BF0209A08202805C298024BECD4
:104B6700C29A7884E60624AEF582E4340CF583E530
:104B770099F0C298E6FFB40112900CAEE0FE700304
:104B8700F68066EE54072402788BF6EFB4020D78B0
:104B97008BE6B40907900CAFE02403F67884E6FFB0
:104BA700B4400476008042EFC3788B96403B78840C
:104BB700E624FFFDE434FFFC7B017A0C79AE125347
:104BC700897884E624ADF582E4340CF583E06F60E0
:054BD7000476008014CB
:0D4BDC0075261475271300D527FCD526F685
:104BE90012260278847600D007D006D005D004D0EA
:104BF90003D002D001D000D0D0D082D083D0F0D061
:024C0900E03297
:10002600900CAFE075F020A4AB08250AF9E5093578
:10003600F0FA90000D120A97788AE6FF18E68FF01C
:10004600A4252AF582E435F0F583120799FF7B0093
:040056007A0079288B
:10005A008F378B388A39893AE4F584EA494B601C30
:10006A00AB38AA39A93A120780FFE537FD7C00129E
:0C007A005EDCAB38AA39A93AEF1207C6C9
:0D008600753B14753C1300D53CFCD53BF6D2
:0E0093008537997F01125C873099FDC2992252
:095E0000E4F5847881EFF6D28507
:0D5E090075371475381300D538FCD537F601
:075E1600900CEEE0F599226B
:105B1D00C9EFC9E964017028EDC39B4034786CE688
:105B2D00FFEB2FFFE433FEEDC39FEE6480F874802E
:105B3D0098501ED228C3ED9B788AF678867601227E
:105B4D00B90214ED6B700AD228788AF6788676023F
:085B5D0022C228E47886F6223A
:1056EA00C9EFC9BAFF15BBFF12ED6B7002EC6A7005
:1056FA0049D228788AF67886E9F622E96401702583
:10570A00C3ED9BEC9A401C786CE62BFFE43AFEC38F
:10571A00ED9FEC9E500DD228C3ED9B788AF67886D1
:10572A007601228015B90218ED6B7002EC6A700AD4
:10573A00D228788AF67886760222C228E47886F613
:01574A00223C
:10260200900CAEE0FF54F8F529E4F584EF120AC706
:10261200264F09265C0A266F102678112689122673
:10262200A01926B61A26DB2026E428276529286762
:102632003328A23728D13928EB4128F649290050FE
:1026420029486128317029409800002978900CAF00
:10265200E0FD788DE6FB7F018027900CAFE0FCA3C4
:10266200E0FD788CE6FA08E6FB7F01802BD2287821
:10267200867603022978900CAFE0FD788FE6FB7F27
:1026820002125B1D022978900CAFE0FCA3E0FD78FA
:102692008EE6FA08E6FB7F021256EA022978900CCF
:1026A200AFE0FD788DE6FB7F01125B1D202803025F
:1026B2002978801A900CAFE0FCA3E0FD788CE6FA52
:1026C20008E6FB7F011256EA202803022978900CC3
:1026D200EE7478F07F01022975E4F58475EF10023B
:1026E2002978C2ACE4F528D285FB7A0079287F7F6D
:1026F20012005A7B007A0079287F1812005A7B0058
:102702007A0079287F0512005A7882E612005378FF
:102712008CE6120053788DE6120053788EE6120092
:1027220053788FE61200537890E61200537891E6C0
:10273200120053E4F52A7492252AF8E61200530592
:102742002AE52AC3941040EE7B007A007900AF2874
:0327520012005A18
:0D27550075350A75361300D536FCD535F6FE
:1027620002281C900CAFE0FFC37882964003022837
:1027720023EF75F020A4250AF9E50935F085083222
:10278200F5338934C2ACE4F528D285FB7A00792886
:102792007F7F12005A7B007A0079287F0D12005A3F
:1027A200AB32AA33A934120780120053AB32AA33D8
:1027B200A934900001120050AB32AA33A934900020
:1027C20002120050AB32AA33A93490000312005017
:1027D200AB32AA33A934900004120050E4F52AABBC
:1027E20032E5342405F9E43533FA7E00E9252AF985
:1027F200EE3AFA120780120053052AE52AC394081A
:0D28020040DD7B007A007900AF2812005AFB
:0D280F0075350A75361300D536FCD535F643
:10281C00C285D2AC022978900CEE7478F0E4A3F067
:10282C007F02022975125F11780F120A25900CEEA7
:10283C00747CF0780FE6A3F008E6A3F008E6A3F0AA
:10284C0008E6A3F07C007D057B017A0C79EE12532F
:10285C0089900CF3EFF07F06022975900CAFE0FF26
:10286C00B4010FA3E0FDA3E0788CCDF608EDF602E1
:10287C002940EFB4020A900CB0E0788CF6022940A3
:10288C00900CAFE0B4030CA3E0FFA3E0788ECFF67E
:10289C0008EFF6022940E4F52A900CAFE0FFE52A98
:1028AC00C39F501B74B0252AF582E4340CF583E0E9
:1028BC00FF7492252AF8EFF6052AE52AB410DAE41B
:1028CC0078A1F6806F7A007B327D01788AE6FF1260
:1028DC0055A1900CAFE0FDE4FF12595002297890FD
:1028EC000CAFE024FF9202022978900CAFE024FF99
:1028FC0092018078788AE66005752C02800B202B7B
:10290C0005752C038003752C01900CEE7479F0A3E3
:10291C00E52CF07C007D027B017A0C79EE12538958
:10292C00900CF0EFF07F03125E00E52C6401703C1C
:10293C00D22C8002D226788076F180307A007B32DD
:10294C007D017F001255A1900CEE7479F0900CAFC4
:10295C00E0900CEFF07C007D027B017A0C79EE129A
:10296C005389900CF0EFF07F03125E00E52964A010
:10297C006003022B87900CAEE064A16003022A77FF
:10298C00A3E0C37882964003022A6CAB08AA09A97B
:10299C000AE0FF75F020A4F58285F083120799F503
:1029AC002CEF75F020A429F9EA35F0FA9000041206
:1029BC00079930E237900CAFE01200038F2C900C8B
:1029CC00EE747FF0A3E52CF02402FDE433FC7B01D4
:1029DC007A0C79EE12538974F0252CF582E4340CC0
:1029EC00F583EFF0E52C2403FF022B84900CAFE071
:1029FC00FF120003C2ACE4F528D285E52CD3940673
:102A0C00402B7B007A0079287F7F12005A7B007A5A
:102A1C00007928AF2C12005AE4F52AE52AC3952C2C
:102A2C005007120026052A80F2052C8018E52C246C
:102A3C0078120053E4F52AE52AC3952C50071200AE
:102A4C0026052A80F27B007A007900AF2812005A02
:0D2A5C0075350A75361300D536FCD535F6F4
:102A6900022B76900CEE7478F07F01022B84900C87
:102A7900AEE064A26003022B877882E6FFA3E0FE42
:102A8900C39F4003022B7CA3E0FDC39F4003022B9D
:102A99007CEE9D4003022B7C900CAFE0F52AE4F517
:102AA90030F531900CB0E0FFE52AD39F5026AF2ACC
:102AB900120003AB08AA09A90A75F020E52AA4F5B2
:102AC9008285F0831207992531F531E43530F530E7
:102AD900052A80CFC2ACE4F528D285FB7A00792893
:102AE9007F7F12005AC3E5319480E530940050028B
:102AF9008007E5304480120053AF31120054900C26
:102B0900AFE0F52A900CB0E0FFE52AD39F5046E4E8
:102B1900F52BAB08AA09A90A75F020E52AA4F582C4
:102B290085F083120799FFE52BC39F5024E52A7589
:102B3900F020A429F9EA35F0FA90000D120A9778E5
:102B49008AE6FF18E68FF0A4252B120049052B8091
:102B5900C1052A80AF7B007A007900AF2812005A9C
:0D2B690075350A75361300D536FCD535F6E6
:102B7600C285D2AC800B900CEE7478F07F01125EA9
:102B860000E5296458704DFA7B327D01788AE6FFAC
:102B96001255A1753A01753B0C753CEF7B017A0C19
:102BA60079AF125C5A8F2CE52C2478900CEEF0EF5E
:102BB6002401FDE433FC7B017A0C79EE125389740F
:102BC600EF252CF582E4340CF583EFF0E52C240296
:102BD600FF125E00E52964806009E52964886003C8
:102BE600022D967886E6B4010F7A007B327D017855
:102BF6008AE6FF1255A1801AE4F52AE52AC3786C05
:102C060096500F7A007B327D01AF2A1255A1052A14
:102C160080E9900CAEE05407F52CB4070A752B0139
:102C2600A3E0F52CA38006E4F52B900CAFE0F52D80
:102C3600152CE52DC37882964003022D6AAB08AAAF
:102C460009A90A75F020E52DA4F58285F0831207FF
:102C560099FFE52CD39F40028F2C7886E6B40109B4
:102C6600788AE6F52FF52E8009E4F52E786CE614C1
:102C7600F52F788AA62E788AE6D3952F4003022D63
:102C86005EE4F52AE52AC3952C4003022D53E52D73
:102C960075F020A4AB08250AF9E50935F0FA90008D
:102CA6000412079930E203022D4E90000112079993
:102CB60064387041E52CD394044011E52B252A2471
:102CC600B0F582E4340CF583E0FD805E7884E6C3DB
:102CD600952AFFE49400FE74AC2FF582740C3EF541
:102CE60083E0FDE52D75F020A4AB08250AF9E5097A
:102CF60035F0FA8035AB08AA09A90A75F020E52D4A
:102D0600A4F58285F083120799FFC37884E69F2590
:102D16002A252B24ADF582E4340CF583E0FDE52D60
:102D260075F020A429F9EA35F0FA90000D120A97F9
:102D3600788AE6FF18E68FF0A4FFE52A2FF582E4ED
:102D460035F0F583ED1207D8052A022C8AAF2D122D
:102D5600585A788A06022C7C788AA62EE529648839
:102D6600702E8010E52DB4FF27900CB0E0F520E51D
:102D760029B4881C900CEE7478F07884E624ADF5BE
:102D860082E4340CF583E0900CEFF07F02125E00D3
:012D9600221A
:10F000007880E664F1600302F60CE4F553F5547879
:04F0100081E6601F16
:0DF0140075590A755A1300D55AFCD559F6E6
:10F021000554E5547002055364107004E5536427D8
:10F0310070DCC2AF7584015398FC75FFDE75FFADBE
:10F04100E4F54FF54EE4F58420982EE4F553F5549C
:0EF05100209822C3E5549488E5539413501779
:0DF05F0075590A755A1300D55AFCD559F69B
:10F06C000554E55470DF055380DBB2A080CF859941
:10F07C004EC298E54E641A600302F14CF553F554F8
:0EF08C00209822C3E5549488E553941350173E
:0DF09A0075590A755A1300D55AFCD559F660
:10F0A7000554E55470DF055380DB30989285994FFE
:10F0B700C298E4F553F554209822C3E5549488E5A3
:05F0C7005394135017E3
:0DF0CC0075590A755A1300D55AFCD559F62E
:10F0D9000554E55470DF055380DB20980302F046A0
:10F0E90085994FC298E4F553F554209822C3E55405
:08F0F9009488E55394135017AD
:0DF1010075590A755A1300D55AFCD559F6F8
:10F10E000554E55470DF055380DB20980302F0466A
:09F11E0085994FC298D285C2996F
:0DF12700755914755A1300D55AFCD559F6C8
:06F134007599783099FD89
:0DF13A0075590A755A1300D55AFCD559F6BF
:10F14700C28502F5FEE54E6450600302F1DCF5531B
:10F15700F554209822C3E5549488E5539413501727
:0DF1670075590A755A1300D55AFCD559F692
:10F174000554E55470DF055380DB20980302F04604
:09F1840085994FC298D285C29909
:0DF18D00755914755A1300D55AFCD559F662
:08F19A007599793099FDC299C5
:0DF1A200755914755A1300D55AFCD559F64D
:08F1AF007599013099FDC29928
:0DF1B700755914755A1300D55AFCD559F638
:06F1C400E4F5993099FD0D
:0DF1CA0075590A755A1300D55AFCD559F62F
:0FF1D700C28502F5FEE54E6401703ED285C299F5
:0DF1E600755914755A1300D55AFCD559F609
:08F1F3007599783099FDC2996D
:0DF1FB00755914755A1300D55AFCD559F6F4
:06F20800E4F5993099FDC8
:0DF20E0075590A755A1300D55AFCD559F6EA
:10F21B00C28502F5FEE54E6402600302F2E2F5538D
:10F22B00F554209822C3E5549488E5539413501752
:0DF23B0075590A755A1300D55AFCD559F6BD
:10F248000554E55470DF055380DB20980302F0462F
:10F2580085994FC298E4F550E54F13B392A0E54F56
:10F2680025E0FEC3E49400EE94F0502AE54F7F00B9
:10F2780025E0FEC394E0501EE54F20E01FE4F5842E
:10F2880043B701758F038E558F568F828E83F05347
:10F29800B7F0F58F80037550FFE4F584D285C299E5
:0DF2A800755914755A1300D55AFCD559F646
:08F2B5007599783099FDC299AA
:0DF2BD00755914755A1300D55AFCD559F631
:06F2CA008550993099FD0A
:0DF2D00075590A755A1300D55AFCD559F628
:10F2DD00C28502F5FEE54E6403600302F42DF5537D
:10F2ED00F554209822C3E5549488E5539413501790
:0DF2FD0075590A755A1300D55AFCD559F6FB
:10F30A000554E55470DF055380DB20980302F0466C
:10F31A0085994FC298E4F553F554209822C3E554D1
:08F32A009488E5539413501779
:0DF3320075590A755A1300D55AFCD559F6C5
:10F33F000554E55470DF055380DB20980302F04637
:10F34F00859951C298E54F1392A0E54F25E0FEC372
:10F35F00E49400EE94F0400302F046E54F7D002563
:10F36F00E0FCC394E0400302F046E4F58443B701A8
:10F37F00758F01E55175F020A42DFFE5F03CF55593
:10F38F008F56E4F584F552E552C394205048E4F5C6
:10F39F0053F554209822C3E5549488E553941350A1
:01F3AF001746
:0DF3B00075590A755A1300D55AFCD559F647
:10F3BD000554E55470DF055380DB20980302F046B9
:10F3CD000556E556AE557002055514F5828E83E54A
:10F3DD0099F0C298055280B1E4F58453B7F0F58FDA
:06F3ED00F584D285C299EF
:0DF3F300755914755A1300D55AFCD559F6FA
:08F400007599783099FDC2995D
:0DF40800755914755A1300D55AFCD559F6E4
:06F41500E4F5993099FDB9
:0DF41B0075590A755A1300D55AFCD559F6DB
:10F42800C28502F5FEE54E6404600302F4DDF5537F
:10F43800F554209822C3E5549488E5539413501743
:0DF4480075590A755A1300D55AFCD559F6AE
:10F455000554E55470DF055380DB20980302F04620
:10F4650085994FC298E54F25E0F557755800E4F5A5
:10F4750050F553F5540558E558AE57700205571425
:10F48500F5828E83E4932550F5500554E5547002BA
:0EF4950005537004E553640270DBD285C29902
:0DF4A300755914755A1300D55AFCD559F649
:08F4B0007599783099FDC299AD
:0DF4B800755914755A1300D55AFCD559F634
:06F4C5008550993099FD0D
:0DF4CB0075590A755A1300D55AFCD559F62B
:10F4D800C28502F5FEE54E6405600302F5F3F553B7
:10F4E800F554209822C3E5549488E5539413501793
:0DF4F80075590A755A1300D55AFCD559F6FE
:10F505000554E55470DF055380DB20980302F0466F
:10F5150085994FC298E4F553F554209822C3E554D4
:08F525009488E553941350177C
:0DF52D0075590A755A1300D55AFCD559F6C8
:10F53A000554E55470DF055380DB20980302F0463A
:09F54A00859951C298D285C2993D
:0DF55300755914755A1300D55AFCD559F698
:08F5600075997F3099FDC299F5
:0DF56800755914755A1300D55AFCD559F683
:10F575007599203099FDE54F25E0FCE55175F020A2
:10F58500A42400FFE5F03CF5578F58E4F550F552FB
:02F59500C29919
:0DF59700755914755A1300D55AFCD559F654
:10F5A400855882855783E493F5993099FD0558E58C
:10F5B40058AE577002055714F5828E83E493255094
:0BF5C400F5500552E552B420C8C29972
:0DF5CF00755914755A1300D55AFCD559F61C
:06F5DC008550993099FDF5
:0DF5E20075590A755A1300D55AFCD559F613
:10F5EF00C285800BE54EB40606E4F58475EF10E591
:0DF5FF004E6407600302F0467880F6D2AF3C
:01F60C0022DB
:105269007F00125C87125A8B20270B7A007B327DD4
:10527900017F001255A1302A0B7A007B1E7D017F28
:10528900001255A1302617302B147A007B327D018C
:10529900788AE6FF1255A1C226125090D2272029FA
:1052A9000C302B09788076F1125090D229302C2AB3
:1052B900302B27C22C125ECFE4FDFF125E647BFF08
:1052C9007A5C79B3125D097D01E4FF125E647BFFAC
:1052D9007A5C79C1125D0912F000202B12125F0766
:1052E900E47B2C7A01F9F8C312092E5002D22B2241
:0B5EE80012390512526912412980F89E
:1049E400005EBCE2613FDD83C29C7E20A3FD1F41CB
:1049F4009DC3217FFCA2401E5F01E3BD3E6082DCBB
:104A0400237D9FC1421CFEA0E1BF5D0380DE3C62AA
:104A1400BEE0025CDF81633D7C22C09E1D43A1FF9A
:104A24004618FAA427799BC584DA3866E5BB59078A
:104A3400DB856739BAE406581947A5FB7826C49A7A
:104A4400653BD987045AB8E6A7F91B45C6987A246A
:104A5400F8A6441A99C7257B3A6486D85B05E7B95A
:104A64008CD2306EEDB3510F4E10F2AC2F7193CD4A
:104A7400114FADF3702ECC92D38D6F31B2EC0E503A
:104A8400AFF1134DCE90722C6D33D18F0C52B0EE2A
:104A9400326C8ED0530DEFB1F0AE4C1291CF2D731A
:104AA400CA947628ABF517490856B4EA6937D58B0A
:104AB4005709EBB536688AD495CB2977F4AA4816FA
:104AC400E9B7550B88D6346A2B7597C94A14F6A8EA
:104AD400742AC896154BA9F7B6E80A54D7896B35DA
:104AE400000000002B6096CBDDEE002C96CBDDE5BC
:044AF400EEF7FAFDE2
:105A6700C1AF420C000000420C040000420C0208C7
:095A770000420C06080001AF0A10
:10538900150E150EA80EECF608EDF6150E150E15F0
:105399000EA80EC6EBC608C6EAC608C6E9C6E50EDB
:0453A90024FCF50EDD
:1053AD00F80808E4F6A80EF608F6E50E2407F9A8A5
:1053BD000EE6FE08E6FFC3099719E76480F8EE6470
:1053CD0080985037E50E2404F8CBE6CB08E6FA08B2
:1053DD00E6F98F828E83120799A80E080866FFE5FD
:1053ED000E2403F8EFF6E69049E493A80E0808F6AC
:1053FD00A80E0806E61870B20680AFA80E0808E6DB
:01540D00FF9F
:07540E00E50E2409F50E2252
:0B5EDC00ED6F7813F6E69049E493FFA9
:015EE7002298
:0300A300024DAE5D
:104DAE00C0E0C0F0C083C082C0D0E8C0E0E9C0E07F
:104DBE00EAC0E0EBC0E0ECC0E0EDC0E0EEC0E0EF3A
:104DCE00C0E0E59830E11B900C02E0FEA3E0FF90FE
:104DDE000C06E06E7003A3E06F7002C2845398FD60
:104DEE00D22FE59830E057900C05E02401FF900C8F
:104DFE0004E03400FE900C00E06E7003A3E06F70D0
:104E0E00055398FE8038900C04E475F001120842A8
:104E1E0085F082F583E599F0900C04E06408700447
:104E2E00A3E06400700A900C047400F0A37400F008
:104E3E005398FE7A007B647D017F011255A1D0E06C
:104E4E00FFD0E0FED0E0FDD0E0FCD0E0FBD0E0FAF9
:104E5E00D0E0F9D0E0F8D0D0D082D083D0F0D0E03E
:014E6E003211
:105A8B00900C02E0FEA3E0FF900C06E06E7003A307
:105A9B00E06F6034302F31C22FD284758401900CAB
:105AAB0002E475F00112084285F082F583E0F59966
:105ABB00900C02E0640C7004A3E06400700A900C7C
:095ACB00027408F0A37400F0223B
:1058AC00900C00E0FEA3E0FF900C04E06E7003A3EC
:1058BC00E06F6039900C00E475F00112084285F03D
:1058CC0082F583E0786DF6900C00E064087004A318
:1058DC00E06400700A900C007400F0A37400F0787F
:1058EC006DE6FEB40D037F0A22CFEECF2212526971
:0258FC0080AE7C
:105B6500900C00E0FEA3E0FF900C04E06E7003A330
:105B7500E06F6030900C00E475F00112084285F08A
:105B850082F583E07819F6900C00E064087004A3B0
:105B9500E06400700A900C007400F0A37400F078C3
:065BA50019E6FF227FFF5C
:015BAB0022D7
:0852F9008B498A4A894B8D4C58
:10530100125F077814120A25E47818F6125B65EF2C
:10531100F46037EF640A6032BF0D13AB49AA4AA9A2
:105321004B7818E6FFF582758300E40207D8AB4994
:10533100AA4AA94B7818E606F582758300EF120791
:10534100D87818E6FF654C700122125269125F0786
:10535100ECC0E0EDC0E0EEC0E0EFC0E0AF4DE4FC3A
:10536100FDFE78141209D8EF2BFBEE3AFAED39F96C
:10537100EC38F8D0E0FFD0E0FED0E0FDD0E0FCD387
:0753810012092E50877F0086
:015388002202
:105BAC00900C07E02401FD900C06E03400FC900CF6
:105BBC0002E06C7003A3E06D700122900C06E4759A
:105BCC00F00112084285F082F583EFF0900C06E0AC
:105BDC00640C7004A3E06400700A900C067408F066
:055BEC00A37400F0228B
:105DA300900C02E0FEA3E0FF900C06E06E7003A3EC
:0F5DB300E06F600A7F00125C87125A8B80E22239
:105AD4007E007F00900C04EEF0A3EFF0900C00EE3B
:105AE400F0A3EFF07E087F00900C06EEF0A3EFF039
:105AF400900C02EEF0A3EFF07E087F007D007B01A6
:105B04007A007900120BD67E047F007D007B017A37
:095B1400087900120BD6D22F22F1
:10595000EF7025F5847598D0F584759115F58475EB
:10596000C90875CBFFED904AE393F5CA75C804E406
:10597000F584D2ACC2BC8026758401759850E4F5DC
:1059800084E589540F4420F589758E02ED904AED27
:1059900093F58DD28E43E74043F740125AD4D2AFED
:0159A00022E4
:1059A10078B2120A3D0000000078B6120A3D0000EC
:1059B100000078A27664E47814F67814E6FFC394C4
:1059C10003502DEF25E025E024A3F8E4F6EF25E0D0
:1059D10025E024A4F8E4F6EF25E025E024A5F8E489
:1059E100F6EF25E025E024A6F8E4F678140680CA4F
:0159F1002293
:105DC200D2AFD2A9C2BBE4F584E589540F4401F5F0
:0F5DD20089758E02758CAFE4F58AD28C0259A1C7
:02513300150E57
:10513500A80EE4F6A80EE6FFC3940340030251CC83
:10514500EF25E025E024A6F8E6FFD394004052A819
:105155000EE625E025E024A4F8E67045EF30E015DD
:10516500A80EE6FF25E025E024A6F8E6D394014045
:10517500047D0180067D00A80EE6FF1257A8A80E43
:10518500E6FF25E025E024A6F816E66014EF25E005
:1051950025E024A5F8E6FEEF25E025E024A4F8EEB9
:1051A500F6A80EE625E025E024A4F8E6600116A899
:1051B5000EE6FF25E025E024A6F8E67004FD12576B
:0751C500A8A80E06025139F3
:0351CC00050E22AB
:03000B000254A1FB
:1054A100C0E0C0F0C083C082C0D0E8C0E0E9C0E085
:1054B100EAC0E0EBC0E0ECC0E0EDC0E0EEC0E0EF40
:1054C100C0E0758CAF78B21209BCEF2401FFE43E55
:1054D100FEE43DFDE43CFC78B2120A2578A216E612
:1054E100701B78B61209BCEF2401FFE43EFEE43DD7
:1054F100FDE43CFC78B6120A2578A2766412513399
:10550100125D81D0E0FFD0E0FED0E0FDD0E0FCD024
:10551100E0FBD0E0FAD0E0F9D0E0F8D0D0D082D0F2
:0655210083D0F0D0E0325F
:105D3300150EA80EEDF6150EA80EEFF6A80EE6FF4B
:105D4300C39403500D08E6FEEF25E025E024A3F8F5
:075D5300EEF6050E050E221D
:1055A100150E150EA80EEAF608EBF6150EA80EED6F
:1055B100F6150EA80EEFF6A80EE6FFC3940350529F
:1055C100EF25E025E024A6F8E67047A80EE6FB25C6
:1055D100E025E024A4F8E67039A80E08E625E004E9
:1055E100FFA80EE6FA25E025E024A6F8EFF6A80EBE
:1055F1000808E6FE08E6FF7C007D0A12080CEA2591
:10560100E025E024A5F8EFF6EB25E025E024A4F859
:09561100E4F6E50E2404F50E2276
:1057A800150EA80EEDF6150EA80EEFF6A80EE6FFDC
:1057B800C39403501CEF25E025E024A3F8E660110C
:1057C800A80E08E670047F0180027F00A80E08EF8B
:1057D800F6A80EE6700608E624FF92A0A80EE6FFDB
:1057E800B4010608E624FF9286EFB40208A80E0862
:0A57F800E624FF9287050E050E223D
:095F0700C2AF78B21209BCD2AF9E
:015F1000226E
:095F1100C2AF78B61209BCD2AF90
:015F1A002264
:105C8700150EA80EEFF6A80EE6700578B0F608F622
:105C9700302D1678AFE675F064A4FFC378B1E69FA0
:0C5CA70018E695F0500375FFA5050E22CD
:105DE100D22DE478B0F608F6EF78AF6003F68002C2
:0F5DF100760A75FF0775FFA5E4F58475EF0422A8
:105E7800C22DE478B0F608F678AF76FF75FFDE75C8
:035E8800FFAD2249
:105D810078B106E618700106302D1678AFE675F089
:105D910064A4FFC378B1E69F18E695F0500375FF40
:025DA100A52239
:045CDE008E418F4222
:105CE200E4F543F544C3E5449542E5439541501636
:105CF2007FE87E0312562C7F01125C870544E5443F
:065D020070E3054380DFA1
:015D08002278
:10561A0054F0FFE5A054014FF5A0A21292A37F0116
:02562A007E0000
:04562C008E688F698C
:10563000D3E56994FAE5689400500EEFD3940040E6
:10564000407E1600DEFD1F80F285686A85696BD397
:10565000E56B94FAE56A940040157FFA7E001256D5
:105660002C7406256BF56B74FF356AF56A80E0D300
:10567000E5699400E56894004007AF6BAE6A125686
:015680002CFD
:015681002206
:10568200754C00754D00754E467B007A0079447D5D
:015692000215
:085693008B488A49894A8D4BBE
:10569B007F01125C87AB4CAA4DA94E12085824000F
:1056AB00FFE5F034E0FE85484F854950854A51E4CB
:1056BB00FDEDC3954B501BEF2DF582E43EF583E4D6
:1056CB0093AB4FAA50A9518D827583001207D80D49
:0F56DB0080DFAB4CAA4DA94EE4854BF00208834B
:104F2D00755012755134755800755900755A527B6C
:074F3D00007A0079507D02AB
:084F44008B548A5589568D57E4
:104F4C007880E664F16003024FE1125E78C2AFE450
:104F5C00F58443B701758F01AB58AA59A95A1208A9
:104F6C00582400FFE5F034E07819F608EFF6AA555E
:104F7C00A956781DA65408C6EAC608C6E9C6E47840
:104F8C001BF6781BE6C395575032781DCBE6CB0841
:104F9C000806E618CAE6CA70010614F912078078EA
:104FAC001CF6E6FF78190806E618CCE6CC7001066C
:104FBC0014F5828C83EFF0781B0680C6E4F58F53D2
:104FCC00B7F0AB58AA59A95A8557F0120883D2AF3B
:054FDC00E4FF125DE19D
:014FE10022AD
:1059F2007880E664F17046C2AF125E78E4F58443C3
:105A0200B701758F03781A76E008F67819F6781AD6
:105A1200E6FE08E6F5828E83E4F07F01125C877869
:105A22001BE426F618740236F61806E6C3940840FC
:0D5A3200DDE4F58F53B7F0D2AFFF125DE158
:015A3F002244
:105090001259F2E4F552F553F558755900755A5204
:1050A000FB7A00798C7D16124F44124F2DE4F54F98
:1050B000E54FC3786C965073E4F54EAB08AA09A986
:1050C0000A75F020E54EA4F58285F08312079960F9
:1050D00056E54E75F020A429F9EA35F0FA90000D56
:1050E000120A977889E6854FF0A429F9EA35F0FA93
:1050F000EBC0E0EAC0E0E9C0E0AB08AA09A90A7584
:10510000F020E54EA4F58285F083120799FD7558CD
:1051100000755900755A52D0E0F9D0E0FAD0E0FBA2
:10512000124F44054E8094054F8085124F2DE47830
:0251300080F607
:01513200225A
:034CE500CCEFCC45
:104CE800E4F546F547F543F54C754D00754E46FB22
:104CF8007A00798C7D16125693125682E5456434F3
:104D08007004E54464127003434301EC7003024DE0
:104D1800A8E4F542E542C3786C965073E4F541ABDC
:104D280008AA09A90A75F020E541A4F58285F0834F
:104D38001207996056E54175F020A429F9EA35F083
:104D4800FA90000D120A977889E68542F0A429F9AD
:104D5800EA35F0FAEBC0E0EAC0E0E9C0E0AB08AA47
:104D680009A90A75F020E541A4F58285F0831207A8
:104D780099FD754C00754D00754E46D0E0F9D0E0B0
:104D8800FAD0E0FB125693054180940542808512C3
:104D98005682E54564347004E54464127005800069
:054DA800434302AF438C
:014DAD0022E3
:02574B008F6667
:10574D00302E5743A0F075840F75A60FC2A3D2A2B9
:10575D00125628D2A1E4F5677F0A7E0012562C302E
:10576D00A7090567E567C394C840EDC2A112562885
:10577D00C2A275840F75A6FF125628E56612561A39
:10578D00D2A1125628C2A1125628E566C412561A85
:0A579D00D2A1125628C2A11256280C
:0157A70022DF
:105C2A008F4153A00FE54154F042A0D2A112562849
:105C3A00C2A112562853A00FE541C454F042A0D283
:105C4A00A1125628C2A11256287F647E0002562C41
:10552700E47814F608F6C2A1C2A2C2A375840F7567
:10553700A6FF53A00143A020D2A17F01FE12562C43
:10554700C2A17F017E00125CDE7F20125C2A43A08D
:10555700F075840F75A60FC2A3D2A2125628D2A146
:105567007F647E0012562C30A703C22E22D22EC291
:10557700127F2412574BC2127F0B12574BC2127F56
:105587002012574BC2127F0C12574BC2127F0112C7
:09559700574BC2127F0612574B5C
:0155A00022E8
:0D5ECF00C2127F0112574BE4FDFF025E641A
:105EAF00EF6006C2127F0F8004C2127F0C12574B95
:015EBF0022C0
:105E6400ED5403C43354E0FEEF541F44804EFFC28C
:045E74001202574B74
:105E39008F65E565640D600BE565640A6005D2123E
:065E490012574BAF652269
:105D5A008B0B8A0C890DAB0BAA0CA90D120780605C
:105D6A0015050DE50D7002050C14F9120780FFD216
:075D7A001212574B80E022DA
:103EDB00202020202020202020200025622A626420
:103EEB000025622A62750025622A640025622A7504
:103EFB000025622A2E622A660025622A6C64002540
:103F0B00622A6C7500253262753A257300202020D9
:103F1B002020202020004E6F207661726961626C38
:103F2B00657320646566696E65640020202020201F
:103F3B002020202020202020202020202020004571
:103F4B00534320454E5445522020202D2020202025
:103F5B002B20200045534320454E54455220202012
:103F6B002D20202020202B200045534320454E544C
:103F7B004552202020004553432020202020202084
:103F8B002020002020202020002000506172616D35
:103F9B006574657273207772697474656E00746FE3
:103FAB0020666C617368206D656D6F72792E00F4FD
:103FBB0070000000F76E000000FA8F000000FD6D2E
:103FCB000000000000000000036B000000064D0025
:103FDB00000009470000000C540000000000000026
:103FEB0000016D0000000267000000037300000079
:103FFB00046D00000005680000000641000000078A
:10400B004B00000008804300000980460000144864
:10401B007A0000155061000016626100001757000E
:10402B000000185600000019B50000001A540000DB
:10403B00001B6C2F73001C52504D001D46000000DE
:10404B001E4A0000005A250000005B52504D005CD8
:10405B00636E74005D780000000000000000023504
:10406B000000004E6F64652041647200008C0000FC
:10407B000000003F8000000000000000000002353F
:10408B00000000477270204164720000008E000037
:10409B000000003F800000000000000000000A3814
:1040AB0000000054696D6500000000010DBC0000AC
:1040BB000000003F800000000000000000000A38F4
:1040CB000000004461746500000000010DAC0000AD
:1040DB000000003F800000000000000000000032E4
:1040EB00000004466C6173680000000000000000D3
:1040FB000000000000000000000000000000003283
:10410B000000045265626F6F740000000000000035
:0E411B00000000000000000000000000000096
:0A5A8000C19DC125C124C11EC11F34
:063C0C008B3D8A3E893F5A
:103C120090000112079964387060854046854147DB
:103C2200854248F549754A0A7B017A0D79A01258F6
:103C3200FE7B017A0D79A0125E4FC3EF940AEE6407
:103C42008094805032E4900D55F07B017A0D79A07A
:103C5200125E4FC3740A9FFFE49EFE900D55E0C3AF
:103C62009FEE6480F8748098500D7F20125E399028
:103C72000D55E004F080D3023ED1E4900DA0F0ABEC
:103C82003DAA3EA93F9000021207996066E4900D9A
:103C920055F0900D55E075F005A424BAF582E43490
:103CA2003FF583E493FF6019AB3DAA3EA93F900024
:103CB20002120799FEEF6E6008900D55E004F08045
:103CC200D1900D55E0FF75F005A424BAF582E434D5
:103CD2003FF583E493601CEF75F005A424BBF974EF
:103CE2003F35F07546FFF54789487B017A0D79A08B
:103CF200125802AB3DAA3EA93F90000112079960FB
:103D020066E4900D55F0900D55E075F005A424EC95
:103D1200F582E4343FF583E493FF6019AB3DAA3E9C
:103D2200A93F900001120799FEEF6E6008900D55B1
:103D3200E004F080D1900D55E0FF75F005A424EC6D
:103D4200F582E4343FF583E493601CEF75F005A43B
:103D520024EDF9743F35F07546FFF54789487B013C
:103D62007A0D79A01258027B017A0D79A0125E4F6A
:103D7200900D56EFF0AB3DAA3EA93F1207801460AA
:103D82001D14606424FE7003023E3A2404600302A0
:103D92003ED17BFF7A3E79DB125D09023ED1AB3D1B
:103DA200AA3EA93F900004120799900D5630E11CDB
:103DB200E0FFC3740A9FF54CAB40AA41A942120727
:103DC20080F54D7BFF7A3E79E6023ECEE0FFC3747A
:103DD2000A9FF54CAB40AA41A942120780F54D7BE0
:103DE200FF7A3E79EC023ECEAB3DAA3EA93F90005F
:103DF20004120799900D5630E11FE0FFC3740A9F29
:103E0200F54CAB40AA41A942120858F54E85F04D37
:103E12007BFF7A3E79F2023ECEE0FFC3740A9FF541
:103E22004CAB40AA41A942120858F54E85F04D7B91
:103E3200FF7A3E79F7023ECEAB3DAA3EA93F900003
:103E42000412079930E033900D56E0FFC3740A9FC5
:103E5200F54C900010120799FF600280027F038FD9
:103E62004DAB40AA41A9421209528F518E508D4F3B
:103E72008C4E7BFF7A3E79FC8052AB3DAA3EA93F35
:103E8200900004120799900D5630E121E0FFC374AF
:103E92000A9FF54CAB40AA41A9421209528F508E9B
:103EA2004F8D4E8C4D7BFF7A3F7904801FE0FFC31C
:103EB200740A9FF54CAB40AA41A9421209528F5095
:103EC2008E4F8D4E8C4D7BFF7A3F790A1234F87BF0
:083ED200017A0D79A0125D09CF
:013EDA0022C5
:0D1DF000900D4EE0FBA3E0FAA3E0F97DFFAB
:101DFD008D408B3D8A3E893F9000011207996438D2
:101E0D007003022601AB3DAA3EA93F12078024FEB6
:101E1D00700302206224FE70030222BB24036003C0
:101E2D0002260190000412079920E103021F1CAB4A
:101E3D003DAA3EA93F9000191209F5C000C001C08E
:101E4D0002C003AC40EC1203BBD003D002D001D0D2
:101E5D000012019EC004C005C006C007900D92E09F
:101E6D00FC1203BBD003D002D001D0001200AD1282
:101E7D0003EF900D92EFF0AB3DAA3EA93F900015F8
:101E8D001209729000111209F51203447003022613
:101E9D0001AB3DAA3EA93F900011120972C004C0CA
:101EAD0005C006C007900D92E0FC1203BBA804A963
:101EBD0005AA06AB07D007D006D005D004120344FF
:101ECD005014AB3DAA3EA93F9000111209721203A6
:101EDD00EF900D92EFF0AB3DAA3EA93F9000151289
:101EED000972C004C005C006C007900D92E0FC1237
:101EFD0003BBA804A905AA06AB07D007D006D005D9
:101F0D00D0041203446002500302260102204DE565
:101F1D0040F4704CAB3DAA3EA93F900011120972DE
:101F2D00C004C005C006C007900D92E0FCE412038A
:101F3D00BBA804A905AA06AB07D007D006D005D0CB
:101F4D0004120344701AAB3DAA3EA93F900015122E
:101F5D0009729000111209F5120344600302260163
:101F6D00AB3DAA3EA93F9000191209F5C000C00172
:101F7D00C002C003AC40EC1203BBD003D002D001B1
:101F8D00D00012019EC004C005C006C007900D927E
:101F9D00E0FCE41203BBD003D002D001D00012004C
:101FAD00AD1203EF900D92EFF0AB3DAA3EA93F901D
:101FBD0000151209729000111209F51203447003F5
:101FCD00022601AB3DAA3EA93F900011120972C035
:101FDD0004C005C006C007900D92E0FCE41203BBDF
:101FED00A804A905AA06AB07D007D006D005D004D2
:101FFD001203445014AB3DAA3EA93F9000111209A3
:10200D00721203EF900D92EFF0AB3DAA3EA93F90F7
:10201D000015120972C004C005C006C007900D92CC
:10202D00E0FCE41203BBA804A905AA06AB07D00780
:10203D00D006D005D00412034460025003022601DD
:10204D00AB3DAA3EA93F9000151209721203EF9005
:10205D000D92EFF022AB3DAA3EA93F90000412076E
:10206D009920E1030221609000191209F5C000C00A
:10207D0001C002C003AC40EC1203BBD003D002D0B0
:10208D0001D00012019EC004C005C006C007900D0E
:10209D0092E0FCA3E0FDEC1203B6D003D002D00118
:1020AD00D0001200AD1203EF900D92EEF0A3EFF001
:1020BD00AB3DAA3EA93F9000151209729000111276
:1020CD0009F51203447003022601AB3DAA3EA93F58
:1020DD00900011120972C004C005C006C007900D12
:1020ED0092E0FCA3E0FDEC1203B6A804A905AA0634
:1020FD00AB07D007D006D005D0041203445017AB60
:10210D003DAA3EA93F9000111209721203EF900DE6
:10211D0092EEF0A3EFF0AB3DAA3EA93F9000151251
:10212D000972C004C005C006C007900D92E0FCA363
:10213D00E0FDEC1203B6A804A905AA06AB07D0076B
:10214D00D006D005D00412034460025003022601CC
:10215D000222A3E540F4704FAB3DAA3EA93F90008B
:10216D0011120972C004C005C006C007900D92E09F
:10217D00FCA3E0FDE41203B6A804A905AA06AB076B
:10218D00D007D006D005D004120344701AAB3DAA77
:10219D003EA93F9000151209729000111209F51217
:1021AD0003446003022601AB3DAA3EA93F900019EE
:1021BD001209F5C000C001C002C003AC40EC12030F
:1021CD00BBD003D002D001D00012019EC004C005C7
:1021DD00C006C007900D92E0FCA3E0FDE41203B62B
:1021ED00D003D002D001D0001200AD1203EF900D3C
:1021FD0092EEF0A3EFF0AB3DAA3EA93F9000151271
:10220D0009729000111209F51203447003022601A0
:10221D00AB3DAA3EA93F900011120972C004C00542
:10222D00C006C007900D92E0FCA3E0FDE41203B6DA
:10223D00A804A905AA06AB07D007D006D005D0047F
:10224D001203445017AB3DAA3EA93F90001112094D
:10225D00721203EF900D92EEF0A3EFF0AB3DAA3E9C
:10226D00A93F900015120972C004C005C006C00731
:10227D00900D92E0FCA3E0FDE41203B6A804A905BD
:10228D00AA06AB07D007D006D005D00412034460D0
:10229D00025003022601AB3DAA3EA93F9000151244
:1022AD0009721203EF900D92EEF0A3EFF022AB3D09
:1022BD00AA3EA93F90000412079920E00302237D56
:1022CD00900D92E0F8A3E0F9A3E0FAA3E0FBC000C3
:1022DD00C001C002C003AB3DAA3EA93F9000191238
:1022ED0009F5C000C001C002C003AC40EC1203BB35
:1022FD00D003D002D001D00012019ED003D002D065
:10230D0001D0001200AD900D92120A31AB3DAA3EE4
:10231D00A93F900011120972900D92E0F8A3E0F917
:10232D00A3E0FAA3E0FB1203445012AB3DAA3EA971
:10233D003F900011120972900D92120A31AB3DAA15
:10234D003EA93F900015120972900D92E0F8A3E09E
:10235D00F9A3E0FAA3E0FB12034460025003022646
:10236D0001AB3DAA3EA93F9000151209720225FB53
:10237D00AB3DAA3EA93F90000412079920E103024C
:10238D0024989000191209F5C000C001C002C003C5
:10239D00AC40EC1203BBD003D002D001D00012012F
:1023AD009EC004C005C006C007900D92E0FCA3E0DE
:1023BD00FDA3E0FEA3E0FFEC1203B1D003D002D0E9
:1023CD0001D0001200AD1203EF900D92120A31AB45
:1023DD003DAA3EA93F9000151209729000111209F5
:1023ED00F51203447003022601AB3DAA3EA93F90AE
:1023FD000011120972C004C005C006C007900D92ED
:10240D00E0FCA3E0FDA3E0FEA3E0FFEC1203B1A806
:10241D0004A905AA06AB07D007D006D005D0041233
:10242D0003445015AB3DAA3EA93F9000111209720D
:10243D001203EF900D92120A31AB3DAA3EA93F90C7
:10244D000015120972C004C005C006C007900D9298
:10245D00E0FCA3E0FDA3E0FEA3E0FFEC1203B1A8B6
:10246D0004A905AA06AB07D007D006D005D00412E3
:10247D00034460025003022601AB3DAA3EA93F90E2
:10248D0000151209721203EF0225FBE540F4705599
:10249D00AB3DAA3EA93F900011120972C004C005C0
:1024AD00C006C007900D92E0FCA3E0FDA3E0FEA3E3
:1024BD00E0FFE41203B1A804A905AA06AB07D007F3
:1024CD00D006D005D004120344701AAB3DAA3EA924
:1024DD003F9000151209729000111209F512034474
:1024ED006003022601AB3DAA3EA93F9000191209D7
:1024FD00F5C000C001C002C003AC40EC1203BBD05C
:10250D0003D002D001D00012019EC004C005C00648
:10251D00C007900D92E0FCA3E0FDA3E0FEA3E0FF59
:10252D00E41203B1D003D002D001D0001200AD12DD
:10253D0003EF900D92120A31AB3DAA3EA93F9000D8
:10254D00151209729000111209F51203447003025D
:10255D002601AB3DAA3EA93F900011120972C0049D
:10256D00C005C006C007900D92E0FCA3E0FDA3E0FE
:10257D00FEA3E0FFE41203B1A804A905AA06AB0768
:10258D00D007D006D005D0041203445015AB3DAA98
:10259D003EA93F9000111209721203EF900D921295
:1025AD000A31AB3DAA3EA93F900015120972C00435
:1025BD00C005C006C007900D92E0FCA3E0FDA3E0AE
:1025CD00FEA3E0FFE41203B1A804A905AA06AB0718
:1025DD00D007D006D005D00412034460174015ABC8
:1025ED003DAA3EA93F9000151209721203EF900DFE
:0525FD0092120A3122D8
:105BF1008F3DE92405F9E43AFA78A07C0D7D017E18
:105C0100007F0812075AE4900DA8F0853D4C754DB0
:105C110001754E0D754FA07BFF7A3F79101234F854
:095C21007BFF7A3F7918025D094E
:102D9700301D40E4900D9FF0900D97120A560000E9
:102DA7000000900D9B120A5600000000C220C221AD
:102DB700C222C223E4900D54F0125F07E47B2C7A01
:102DC70001F9F8C312092E4003023495C21DD20837
:102DD700120CD120251EC208120CD1900D54EFF011
:102DE7007003023485D225E064026003023485D281
:102DF70024023485900D4E30241374FFF0A37440E1
:102E0700F0A37469F0900D527405F08013E508F093
:102E1700A3E509F0A3E50AF07882E614900D52F0D5
:102E2700900D52E0FFC394035005E4A3F0801B907C
:102E37000D9FE0FE7002800EEE900D9FB50705E036
:102E470024FE8002E014900D53F07882E67014207F
:102E57002411FDFF125E647BFF7A3F79211234F85B
:102E6700022FB3E4900D51F0900D51E0FDC3940390
:102E77004003022FB3E4FF125E64900D51E0FF9010
:102E87000D53E02FFFE433FE900D9FE07C00B50764
:102E970008ECB506047F1580027F20125E39900D7D
:102EA70051E0FD7F01125E64900D51E0FF900D53DC
:102EB700E02FFFE433FE900D52E0FDD3EF9D7480C9
:102EC700F86E98400C7BFF7A3F79361234F8022F60
:102ED700AA900D51E0FE900D53E0FD2EFFC007EEC6
:102EE700FFED2FFFE433FEEF7805C333CE33CED8A3
:102EF700F9FF900D4EE0FBA3E0FAA3E02FF9EA3EBD
:102F0700FAD007125BF1900D51E0FD7F0A125E6463
:102F1700301E40900D51E0FF900D53E02FFFE4333A
:102F2700FE900D9FE07C00B50729ECB50625EF78EC
:102F370005C333CE33CED8F9FF900D4EE0FBA3E0A7
:102F4700FAA3E02FF9EA3EFA75400175410D754283
:102F570092804D900D51E0FF900D53E02FFFE43329
:102F6700FEEF7805C333CE33CED8F9FF900D4EE090
:102F7700FBA3E0FAA3E02FF9EA3EFAC003C002C0C0
:102F870001900D4EA3E0FAA3E02FF9EA3EFA900074
:102F97000D120A978B408A418942D001D002D00393
:102FA700123C0C900D51E004F0022E6F900D9FE043
:102FB70075F020A430240F2469F9744035F0FA9095
:102FC7000D4E74FF800D250AF9E50935F0FA900DCD
:102FD7004EE508F0A3EAF0A3E9F0301F5A7D03E4B9
:102FE700FF125E647BFF7A3F794A125D09900D9666
:102FF700E075F003A4240DFF900D53E0FE900D9FA4
:10300700E0C39EFD125E6420190A302007C21FE448
:10301700FF125EAF201A0302348530210302348584
:10302700900D96E004F0E064036003023485C21F4C
:10303700FF125EAF023485201E030232027D03E4D5
:10304700FF125E647BFF7A3F795F125D09900D5333
:10305700E0FF900D9FE0C39FFD7F13125E64201970
:103067000A302007C21EE4FF125EAF301A53202138
:1030770050C21EE4FF125EAF900D4EE0FBA3E0FAD4
:10308700A3E0F9120780FF7E00900D4EA3A3E09006
:10309700000D120A97A801AC02AD037B017A0D79E6
:1030A7009212075A302412900D9FE0FF6003B4017B
:1030B70010D226788076F18008900D9FE0FF125895
:1030C7005A301B0F20220C121DF0125F07900D972C
:1030D700120A31301B2D125F07A804A905AA06ABF7
:1030E70007900D97E0FCA3E0FDA3E0FEA3E02446D4
:1030F700FFE43EFEE43DFDE43CFCD312092E400311
:10310700121DF0301B3B125F07A804A905AA06ABE6
:1031170007900D97E0FCA3E0FDA3E0FEA3E024F4F5
:10312700FFEE3401FEE43DFDE43CFCD312092E40E2
:1031370010900D4EE0FBA3E0FAA3E0F97DF7121D16
:10314700FD201B0A900D97120A5600000000301C44
:103157001C202319900D4EE0FBA3E0FAA3E0F97DB4
:1031670001121DFD125F07900D9B120A31301C3AA8
:10317700125F07A804A905AA06AB07900D9BE0FC00
:10318700A3E0FDA3E0FEA3E02446FFE43EFEE43D0A
:10319700FDE43CFCD312092E4010900D4EE0FBA33A
:1031A700E0FAA3E0F97D01121DFD301C3B125F0719
:1031B700A804A905AA06AB07900D9BE0FCA3E0FDB8
:1031C700A3E0FEA3E024F4FFEE3401FEE43DFDE4BA
:1031D7003CFCD312092E4010900D4EE0FBA3E0FA01
:1031E700A3E0F97D09121DFD301C03023485900D03
:1031F7009B120A56000000000234857D03E4FF128B
:103207005E647882E6D394005003302437900D4EE5
:10321700E0FBA3E0FAA3E0F9900019120972E4FBBE
:10322700FAF9F81203444014900D4EE0FBA3E0FABC
:10323700A3E0F990000412079930E2087BFF7A3F78
:10324700797480067BFF7A3F7981125D097F1212BC
:103257005E397BFF7A3F798E125D097F13125E39E3
:103267007BFF7A3F7994125D0920190C302009C23F
:1032770025C224D208120CD1201A0302336B302145
:103287000302336B7882E6D394004061900D4EE0E1
:10329700FBA3E0FAA3E0F9120780FFD39404504D93
:1032A700EF94004048900019120972E4FBFAF9F80C
:1032B7001203445038D21E900D4EE0FBA3E0FAA350
:1032C700E0F9120780FF7E0090000D120A977892AE
:1032D7007C0D7D0112075A900D53E0FF900D9FE082
:1032E700C39FFD7F13125E647F01125EAF30242AF5
:1032F700900D9FE0FF64026004EFB4031DD21FE44A
:10330700900D96F0900D53E0FF900D9FE0C39FFD49
:103317007F0D125E647F01125EAF302437900D9FE0
:10332700E06404702FD226788076F1125ECFE4FD38
:10333700FF125E647BFF7A3F7996125D097D01E497
:10334700FF125E647BFF7A3F79A9125D097FB87E21
:103357000B125CDE30240D900D9FE0B40506E4F5FA
:103367008475EF10301B2A202227900D9FE07012E2
:103377002024077882E614F0800E900D9F7405F0E4
:103387008006900D9FE014F0125F07900D97120AC8
:1033970031301B48125F07A804A905AA06AB07909E
:1033A7000D97E0FCA3E0FDA3E0FEA3E02446FFE4C5
:1033B7003EFEE43DFDE43CFCD312092E401E900D79
:1033C7009FE070122024077882E614F0800E900D9B
:1033D7009F7405F08006900D9FE014F0201B0A9063
:1033E7000D97120A5600000000302408900D517402
:1033F70006F080077882E6900D51F0301C212023DB
:103407001E900D9FE004FF900D51E0FEEF8EF084BB
:10341700900D9FE5F0F0125F07900D9B120A313077
:103427001C3F125F07A804A905AA06AB07900D9BCE
:10343700E0FCA3E0FDA3E0FEA3E02446FFE43EFE9C
:10344700E43DFDE43CFCD312092E4015900D9FE0AE
:1034570004FF900D51E0FEEF8EF084900D9FE5F094
:10346700F0201C0A900D9B120A5600000000301B2A
:103477000D301C0A202407E4900D9FF0D224A219D6
:0E3487009220A21A9221A21B9222A21C922332
:013495002214
:1000A60002045BE86480F8E933E83360110460F029
:1000B600ED33EC337009E8FCE9FDEAFEEBFF2204C0
:1000C60060DED3EB9FEA9EE99DE8C2E78CF0C2F7BB
:1000D60095F0400CE8CCF8E9CDF9EACEFAEBCFFB87
:1000E60012042685D0F05804700320D5B3E80470B6
:1000F600075002B2D502046592D5EC0460F7E4CC51
:10010600C0E0C398F8603B94186008400DD0E0FB4F
:1001160002043DE4FBFAC9FC8028E830E406E4C9A1
:10012600FBE4CAFCE830E305E4C9CACBFCE85407A3
:100136006010F8C3E913F9EA13FAEB13FBEC13FCAE
:10014600D8F130F52FC3E49CFCEF9BFFEE9AFEED51
:1001560099FDD0E0FBEF4E4D4C701222DB030204FA
:1001660062EC2CFCEF33FFEE33FEED33FDED30E7B2
:10017600EB02043DEF2BFFEE3AFEED39FDD0E0FB3E
:1001860050130BBB0003020465ED13FDEE13FEEFE7
:0801960013FFEC13FC02043D11
:10019E00EC4D6011E8497017ED33EC3304600DE45B
:1001AE00FCFFFEFD22E933E8330470F802045B1213
:1001BE00042658046009E4CC248150062850090214
:1001CE000465284003020462C0E0EB4A7044B98023
:1001DE0006D0E0FB020451EF4E701CBD8008EBFF11
:1001EE00EAFEE9FD80EBE98DF0A4FEE5F002028760
:1001FE00E9CDF9EAFEEBFFEF89F0A4FCE5F0CE893C
:10020E00F0A42EFFE435F0CD89F0A42DFEE435F0F8
:10021E008067EF4E7005BD80D780C3EF8BF0A4AC26
:10022E00F0EE8BF0A42CFCE435F0F8EF8AF0A42C61
:10023E00E5F038FCE433CB8DF0A42CFCE5F03BF874
:10024E00EE8AF0A42CFCE5F038F8E433CF89F0A464
:10025E002CFCE5F038CF3400CE89F0A42FFFE5F06A
:10026E003EFEE433C98DF0A42EFEE5F039CD8AF0C2
:10027E00A42FFFE5F03EFEE43DFD33D0E0FB50073A
:10028E000BBB000F020465EC2CFCEF33FFEE33FECC
:06029E00ED33FD02043DFA
:1002A400020465EC5D046005E85904700302045B14
:1002B400120426580460F6EC4860F2EC7004FDFE6B
:1002C400FF22C860DB2481C85009C398600250062D
:1002D4000204629850CAF582E9294B4A7005AB8240
:1002E40002045175F0007C1A7880C3EF9BEE9AEDFE
:1002F40099400DC3EF9BFFEE9AFEED99FDE842F0A5
:10030400DC23ACF0D0E0FFD0E0FED0E0FDAB8220F7
:10031400E7101BEB60BAEC2CFCEF33FFEE33FEED81
:1003240033FD02043DE803F830E705C0F075F00042
:10033400EF2FFFEE33FEED33FD40B830E7C280AA65
:1003440074F8CC6480CCC86480C8F582046043C36C
:10035400EB9FF5F0EA9E42F0E99D42F0E89C45F0FF
:1003640060305018E5825FFFE582F42B5582FB5024
:10037400210ABA001D09B90019088016E5825BFB41
:10038400E582F42F5582FF50090EBE00050DBD0015
:10039400010CC3EB9FF5F0EA9E42F0E99D42F0E8C0
:0D03A4009C45F06007CC4820E701B3EC2237
:1003B10075F020800E75F010800575F0087D007EC7
:1003C100007F003392D530D50312090AEC33401077
:1003D100EF33FFEE33FEED33FDEC33FCD5F0ED22D0
:0E03E100E5F0247EA2D513CC92E7CDCEFF220C
:1003EF00EDD2E7CD33EC3392D524814006E4FFFE06
:1003FF00FDFC22FCE4CFCECDCC24E0501174FF8065
:10040F00EDC3CC13CCCD13CDCE13CECF13CF047001
:07041F00F030D5DE02090AEE
:10349600E560244CF8E60560227849301002784C45
:1034A600E475F001120A870207802009EB7F2ED20D
:1034B600098018EF540F2490D43440D4FF300D0BFC
:1034C600EF24BFB41A0050032461FFE561600215C2
:1034D600610564E5647002056330100D7849E47592
:1034E600F001120A87EF0207C6025E397403D21092
:1034F6008003E4C210F5608B498A4A894BE4F56182
:10350600F563F564E56160077F201234D180F575B7
:1035160062FFC20AC209C20BC20CC20EC20FC2119E
:1035260012349FFF700D3010057F001234E2AF6435
:10353600AE6322B4255FC2D5C20D12349FFF24D0DC
:10354600B40A00501A75F00A786130D50508B6FF3E
:103556000106C6A426F620D5047002D20C80D92412
:10356600CFB41A00EF5004C2E5D20D0237CFD20A0B
:1035760080C6D20980C0D20B80BCD2D580BAD20E0A
:1035860080B47F201234D1200B077401B56100404E
:10359600F1123496FF1234D102350AD211D20F80BD
:1035A60095123496FB123496FA123496F94A4B70F9
:1035B6000679C67A387BFF200B2EE561602A7E00ED
:1035C6008E8275830012079960060EEE656270F0B2
:1035D600C2D5EBC0E0EAC0E0E9C0E0EE12382FD079
:1035E600E0F9D0E0FAD0E0FB120780FF60AAEBC05A
:1035F600E0EAC0E0E9C0E01234D1D0E02401F9D01D
:10360600E03400FAD0E0FBE5620460DCD562D980E4
:1036160087D20B80A212381260F7E562700104129D
:10362600049BA962600DE562600914F5621238B95F
:10363600EF60F3EA30E702F404C3995077EAF42521
:10364600620430E701E404F562800D12381260C1AD
:10365600EA0562256212049BEA785FF630E701E428
:10366600256204D56204200E011412382FE4C0E04E
:103676001238B9785FE6601320E70714F61234B9FA
:10368600802204F6D0E014C0E07F001234B9E5626F
:1036960060071234B01562800B300E031234B0D0BE
:1036A600E002350AD0E00480C512381260A0E56257
:1036B6000412049B785FEAF6E562200E02600104BC
:0536C600240412382F5E
:1036CB0074FF04C0E01238B91234B9E562200E025F
:1036DB0060031234B0D0E0B562E87F451234C37892
:1036EB005FE67F2B30E7047F2DF404C0E01234D16A
:1036FB00D0E075F00A84C0F01234BAD0E01234BABC
:10370B0002350A791080027908C20FC2118008D2E3
:10371B00D5790A8004790AC2D5E562047002F56294
:10372B00E4FAFDFEFF123496FC7B08200A131234D8
:10373B0096FD7B1030090A123496FE123496FF7BED
:10374B0020EC3382D592D55013C3E43009069FFF8A
:10375B00E49EFEE4200A039DFDE49CFCE4CBF8C24E
:10376B000AEC700CCFCECDCCE824F8F870F38017B0
:10377B00C3EF33FFEE33FEED33FDEC33FCEB33FBEA
:10378B00994002FB0FD8E9EB300A05F8D0E0C448AA
:10379B00B20AC0E00AEC4D4E4F78207B0070C2EAB3
:1037AB00B5620040BCC0E0123831D0F0D0E0200A46
:1037BB0004C4C0E0C4B20AC0F01234BAD0F0D5F0E1
:1037CB00EB02350A120AC735A753370E5835784C1A
:1037DB0035744237124F371A44371A49358D4337F0
:1037EB00205536514636AF45361B4738E650357CAB
:1037FB002D35802E35A32B35842335A12038CF2AA8
:10380B00353C480000359BE562B4FF037562061238
:10381B003496FC123496FD123496FE123496FF78D1
:10382B00580204CA790AA2D5200C14300E09B9101B
:10383B00020404B9080104A2D5200F025001042090
:10384B000B68920BB561005034C0E07F20300C192F
:10385B007F30A20B720F720E500F123888C20BC240
:10386B000FC20EC2117F30800F300E03E9C0E01281
:10387B0034D1300E03D0E0F9D0E0B561CC300E1767
:10388B007F30B9100C1234D17F58300D077F788000
:10389B0003B908031234D1300B057F2D0234D17FCD
:1038AB00202011F87F2B200FF322920B80CF7F006B
:1038BB00B4070050052458F8E6FF22286E756C6C8F
:1038CB002900D20A123496300AF8C20A786130D530
:1038DB000108F602353C2D50434958123496240307
:1038EB00B405004001E49038E1931234C2743A12EB
:0A38FB0034C2D20C75610402370ECE
:1047B7008F408E3F8D3E8C3DE4FFFE7D807C3FAB7E
:1047C70040AA3FA93EA83D1203447009AF40AE3F3F
:1047D700AD3EAC3D22AF40AE3FAD3EAC3D120470A6
:1047E700FBAF44AE43AD42AC41120470FFBF0108BA
:1047F700E4FFFE7D807C3F22EF64046022EB6404CB
:10480700601DBB0127E4FFFEFDFCAB44AA43A942A0
:10481700A84112034460084006E4FFFEFDFC227431
:10482700FFF544F543F542F5410248C5E4F545F582
:1048370046FFFEFDFCAB40AA3FA93EA83D1203443C
:10484700504BAF44AE43AD42AC411203EF8E458FA0
:1048570046AC45AD46EC1203B6C8ECC8C9EDC9CAAB
:10486700EECACBEFCBAF44AE43AD42AC411200A989
:10487700E4FBFAF9F812034470A5AF40AE3FAD3E32
:10488700AC3D12048A8F408E3F8D3E8C3DAF40AECB
:104897003FAD3EAC3D1246B6AB44AA43A942A84140
:1048A70012019E1252078F448E438D428C41E5467A
:1048B70030E00B12048A8F448E438D428C41AF4403
:0748C700AE43AD42AC4122FB
:10042600E9D2E7C933E833F892D5EDD2E7CD33EC1C
:0704360033FC5002B2D52295
:10043D00EC30E7100FBF000C0EBE00080DBD000420
:10044D000BEB6014A2D5EB13FCED92E7FD2274FFCC
:10045D00FCFDFEFF22E480F8A2D574FF13FC7D8025
:03046D00E480EF39
:10047000ED33EC33601004700FED547F700574029F
:0A04800092E2227404220422E42216
:10048A00ED33EC33600A047003BD8004ECB2E7FC80
:01049A00223F
:10049B00F920E72824F950037907E4F42402FB1828
:1004AB00DBFDE624FB5014E9600DE4F618E604F6D8
:0F04BB00B40A08E4F6D9F57401F60A22C2D52274
:1004CA00ED33EC3392D5FA602AB4FF33EDC2E77B01
:1004DA00FF60067A0479EFE4227A0479F820D504D9
:1004EA007A0479F3224E614E002B494E46002D497B
:1004FA004E4600E47A08F608DAFC7B00740722E824
:10050A00C0E0ECC0E0EDC0E0EEC0E0EFC0E0EA75AC
:10051A00F010A4CAABF075F04DA42BFBE435F0FC47
:10052A00EA2410FAEB34C5FBEC34D9FCEDC2E7FF40
:10053A0075F056A4F42411C5F0F434C58FF0A42A3A
:10054A00E5F03BE43CF620E7141205FDD0E0FFD0CD
:10055A00E0FED0E0FDD0E0FC1202A78014F4041201
:10056A0005FDD0E0FFD0E0FED0E0FDD0E0FC1201B6
:10057A009ED0E0F8E6FAEDD2E7CD33EC332482FBE5
:10058A00E4C3CF33CFCE33CECD33CD33DBF37B07CA
:10059A0075F00A846004F6081B0AE5F0F6088FF085
:1005AA00740AA4FFACF08EF0740AA42CFEACF050CE
:1005BA00010C8DF0740AA42CFDE435F0F608DBDE9C
:0305CA0074072291
:1051CF0033DA929E35B16011377FE5FE392184893C
:1051DF003AAEC3FF3C1D955B3D6358473E75FDF0EE
:1051EF003F3172183F800000C2D502046502045B94
:1051FF00BD80FA50F3020462ED33EC330460F17BAF
:10520F003B7AAA79B8783F12019EED33EC3392D5F1
:10521F00247B5011A2D570DB500BED448024045039
:10522F0004A2D580CEEFFBEEFAEDF9ECF81203EF06
:10523F00EFF582F404FC1203BB1200ADC082905153
:10524F00CF740912064CED33CC33D0F092D525F044
:0A525F00A2D57001C313CC13FD2289
:104682003E9248DA3ECCCCCD3F2AAAAB4000000095
:104692003F8000003F9837F03FB504F33FD744FC1A
:1046A2003E3172173EB172173F0515913EDE5BD95E
:1046B200D2088002C208EDD2E7F8CD33EC330470A1
:1046C2000BBD800592D502046502045B40FBD31446
:1046D20060F2F5F07C3FEE7A00C39496C8948B406A
:1046E200230AC89469C8941A401A0AC89468C894DC
:1046F2001F40110AC8945AC89425400805F07A0050
:10470200CDC2E7CDC0F08C478D488E498F4AEA234F
:1047120023C0E02492F582E43446F5831209E512BF
:1047220000ADECC0E0EDC0E0EEC0E0EFC0E0120989
:10473200C8A847A948AA49AB4A1200A9D0E0FBD0B1
:10474200E0FAD0E0F9D0E0B2E7F81202A78C478D88
:10475200488E498F4A904682740312063DA847A9A3
:1047620048AA49AB4A12019ED0E0600F249EF5820E
:10477200E43446F5831209E51200AD8C478D488E6C
:10478200498F4AD0E0C3947FFDE49400FC1203B643
:104792007B187A727931783F12019EA847A948AAFC
:1047A20049AB4A1200AD30080B7BD97A5B79DE78CF
:0547B2003E12019E22F1
:1005CD003F8000004120000042C80000447A000036
:1005DD00461C400047C35000497424004B189680B8
:1005ED004CBEBC205A0E1BCA6753C21C749DC5AEAF
:1005FD00FB60065407601C232312062BEB54386056
:10060D000912061712062612019EECF8EDF9EEFA04
:10061D00EFCB22EB12062680F1543803241C9005F3
:10062D00CDFE93FC0EEE93FD0EEE930ECE93FF22B8
:10063D00C0E0EFFBEEFAEDF9ECF812019ED0E0F51B
:10064D00F0EFFBEEFAEDF9ECF81209C8A3A3A3A3A2
:10065D00E8C0E0E9C0E0EAC0E0EBC0E0C0F01201A4
:10066D009E1209E5A3A3A3A31200ADD0F0D0E0FB29
:0D067D00D0E0FAD0E0F9D0E0F8D5F0D422BA
:0300000002541592
:0C541500787FE4F6D8FD7581B902545C84
:10068A00E709F608DFFA8046E709F208DFFA803E52
:10069A0088828C83E709F0A3DFFA8032E309F6083F
:1006AA00DFFA8078E309F208DFFA807088828C83A7
:1006BA00E309F0A3DFFA806489828A83E0A3F6085B
:1006CA00DFFA805889828A83E0A3F208DFFA804C35
:1006DA0080D280FA80C680D4806980F2803380100C
:1006EA0080A680EA809A80A880DA80E280CA803375
:1006FA0089828A83ECFAE493A3C8C582C8CCC583ED
:10070A00CCF0A3C8C582C8CCC583CCDFE9DEE780BC
:10071A000D89828A83E493A3F608DFF9ECFAA9F03B
:10072A00EDFB2289828A83ECFAE0A3C8C582C8CC91
:10073A00C583CCF0A3C8C582C8CCC583CCDFEADEAA
:10074A00E880DB89828A83E493A3F208DFF980CC0C
:10075A0088F0EF60010E4E60C388F0ED2402B40405
:10076A000050B9F582EB2402B4040050AF232345AC
:06077A0082239006DA73F1
:10078000BB010689828A83E0225002E722BBFE0277
:09079000E32289828A83E49322AA
:10079900BB010CE58229F582E5833AF583E0225015
:1007A90006E92582F8E622BBFE06E92582F8E2225F
:0D07B900E58229F582E5833AF583E4932279
:1007C600BB010689828A83F0225002F722BBFE0112
:0207D600F3220C
:1007D800F8BB010DE58229F582E5833AF583E8F057
:1007E800225006E92582C8F622BBFE05E92582C803
:0207F800F222EB
:1007FA00EF8DF0A4A8F0CF8CF0A428CE8DF0A42E13
:02080A00FE22CC
:10080C00C2D5EC30E709B2D5E4C39DFDE49CFCEE07
:10081C0030E715B2D5E4C39FFFE49EFE120C02C371
:10082C00E49DFDE49CFC8003120C0230D507C3E46C
:06083C009FFFE49EFE2276
:10084200A3F8E0C5F025F0F0E58215827002158369
:06085200E0C838F0E822C6
:10085800BB010A89828A83E0F5F0A3E0225006876B
:10086800F009E71922BBFE07E3F5F009E31922892D
:0B087800828A83E493F5F07401932260
:10088300BB010789828A83020C57500B09C5F027E5
:10089300F7C5F01937F722BBFE0D09F8E325F0F38E
:1008A300C5F019E338F322F889828A83740193250A
:0808B300F0C5F0F8E4933822CF
:1008BB00E88FF0A4CC8BF0A42CFCE98EF0A42CFCDC
:1008CB008AF0EDA42CFCEA8EF0A4CDA8F08BF0A45A
:1008DB002DCC3825F0FDE98FF0A42CCD35F0FCEBB9
:1008EB008EF0A4FEA9F0EB8FF0A4CFC5F02ECD397E
:0F08FB00FEE43CFCEAA42DCE35F0FDE43CFC22EB
:0E090A00C3E49FFFE49EFEE49DFDE49CFC22FE
:10091800EB9FF5F0EA9E42F0E99D42F0EC6480C856
:0609280064809845F022F6
:10092E00EB9FF5F0EA9E42F0E99D42F0E89C45F01F
:01093E002296
:10093F00E8600FECC313FCED13FDEE13FEEF13FF96
:03094F00D8F122BA
:10095200BB010789828A83020C6D5005E9F80209FE
:10096200BCBBFE05E9F8020C7989828A830209C8B8
:10097200BB010DE58229F582E5833AF583020C6D10
:100982005007E92582F80209BCBBFE07E92582F877
:10099200020C79E58229F582E5833AF5830209C8DA
:1009A200BB010789828A83020A315005E9F8020AEB
:0A09B20025BBFE05E9F8020C9E22A9
:0C09BC00E6FC08E6FD08E6FE08E6FF2267
:1009C800E493FC740193FD740293FE740393FF2275
:0D09D800E6FB08E6F908E6FA08E6CBF8228F
:1009E500E493F8740193F9740293FA740393FB2268
:1009F500BB010DE58229F582E5833AF583020C8575
:100A05005007E92582F80209D8BBFE07E92582F8D7
:100A1500020C91E58229F582E5833AF5830209E521
:0C0A2500ECF608EDF608EEF608EFF622FD
:0C0A3100ECF0A3EDF0A3EEF0A3EFF02238
:100A3D00D083D082E493F608740193F60874029380
:090A4D00F608740393F6740473B7
:100A5600A8828583F0D083D082120A6D120A6D12A5
:100A66000A6D120A6DE473E493A3C583C5F0C583CA
:100A7600C8C582C8F0A3C583C5F0C583C8C582C8EA
:010A8600224D
:100A8700FAE6FB0808E6F925F0F618E6CA3AF62270
:100A9700BB010DE58229F582E5833AF583020CB3A4
:100AA7005007E92582F8020CAABBFE07E92582F860
:100AB700020CBCE58229F582E5833AF583020CC571
:100AC700D083D082F8E4937012740193700DA3A3BE
:100AD70093F8740193F5828883E4737402936860D2
:060AE700EFA3A3A380DFD2
:105D0900120780601CFF09E970010AC0E0EAC0E0DF
:105D1900EBC0E0125E39D0E0FBD0E0FAD0E0F980C8
:0A5D2900DF7F0A125E39E4FEFF225C
:105802008B438A4489458B498A4A894BAB43054578
:10581200E545AA447002054414F912078070ED743C
:10582200FF2545F54574FF3544F544AB460548E58B
:1058320048AA477002054714F9120780FFAB4305D7
:1058420045E545AA447002054414F9EF1207C670F3
:08585200DAAB49AA4AA94B2276
:100AED00E709F60870FA8046E709F20870FA803EC9
:100AFD0088828C83E709F0A370FA807EE309F608FB
:100B0D0070FA8076E309F20870FA806E88828C8321
:100B1D00E309F0A370FA806289828A83E0A3F60864
:100B2D0070FA805689828A83E0A3F20870FA804AAF
:100B3D0080D280FA80C680D4806580F280318010AA
:100B4D0080A680EA809A80A880DA80E280CA80310F
:100B5D0089828A83ECFAE493A3C8C582C8CCC58385
:100B6D00CCF0A3C8C582C8CCC583CC70E9800D89F3
:100B7D00828A83E493A3F60870F9ECFAA9F0EDFBF1
:100B8D002289828A83ECFAE0A3C8C582C8CCC583CA
:100B9D00CCF0A3C8C582C8CCC583CC70EA80DD89F2
:100BAD00828A83E493A3F20870F980CE88F0ED2455
:100BBD0002B4040050C4F582EB2402B4040050BA10
:090BCD002323458223900B3D73A4
:1058FE008B438A448945E4F54BF54CE54A154AAE8F
:10590E0049700215494E6033AB46AA47A9481207A3
:10591E0080FFAB43AA44A945054CE54CAC4B700245
:10592E00054B14F5828C83EF1207D8EF60CD74010E
:10593E002548F548E43547F54780C0AB43AA44A94E
:02594E004522F0
:105E4F00E4FFFE120780600C0FEF70010E09E9707E
:055E5F00F20A80EF22B1
:105E1D00E94A4B700122120780FF6D700122EF706D
:0C5E2D0004FBFAF92209E970ED0A80EA92
:104FE2008B428A438944AB42AA43A944120780FFF9
:104FF200125E8B500D74012544F544E43543F543AC
:1050020080E4D208AB42AA43A944120780FF642B72
:105012006004EFB42D1BAB420544E544AA43700281
:10502200054314F9120780642D6003D38001C392F3
:1050320008E4F545F546AB42AA43A944120780FFAE
:10504200125EC05036AB42AA43A944120780FF3316
:1050520095E0FEEF24D0FBEE34FFFAAE45AF467C7E
:10506200007D0A1207FAEF2BF546EE3AF545740178
:105072002544F544E43543F54380BB300806AE458C
:0E508200AF468009C3E49546FFE49545FE2243
:100BD600EF4E6012EF60010EEDBB010B89828A8336
:100BE600F0A3DFFCDEFA2289F05007F709DFFCA943
:0C0BF600F022BBFEFCF309DFFCA9F0229A
:10542100025EE8E493A3F8E493A34003F68001F25B
:1054310008DFF48029E493A3F85407240CC8C3338C
:10544100C4540F4420C8834004F456800146F6DF5B
:10545100E4800B0102040810204080905A40E47E51
:10546100019360BCA3FF543F30E509541FFEE49350
:10547100A360010ECF54C025E060A840B8E493A317
:10548100FAE493A3F8E493A3C8C582C8CAC583CA42
:10549100F0A3C8C582C8CAC583CADFE9DEE780BEFA
:015A8A00001B
:100C0200BC000BBE0029EF8DF084FFADF022E4CCD6
:100C1200F875F008EF2FFFEE33FEEC33FCEE9DEC9F
:100C2200984005FCEE9DFE0FD5F0E9E4CEFD22EDE5
:100C3200F8F5F0EE8420D21CFEADF075F008EF2F2F
:100C4200FFED33FD4007985006D5F0F222C398FD20
:050C52000FD5F0EA22BD
:100C5700C5F0F8A3E028F0C5F0F8E5821582700228
:060C67001583E038F022C5
:0C0C6D00E0FCA3E0FDA3E0FEA3E0FF22FA
:0C0C7900E2FC08E2FD08E2FE08E2FF22B7
:0C0C8500E0F8A3E0F9A3E0FAA3E0FB22F2
:0D0C9100E2FB08E2F908E2FA08E2CBF822E3
:0C0C9E00ECF208EDF208EEF208EFF22292
:090CAA00E6FB08E6FA08E6F9226F
:090CB300E0FBA3E0FAA3E0F92242
:090CBC00E2FB08E2FA08E2F92269
:0C0CC500E493FB740193FA740293F9228B
:0F5EC000EFC394304007EF943A50028001C322A1
:105E8B00EFC394094005EF940E4003BF2003D3806A
:035E9B0001C3221E
:00000001FF
